:020000040000FA
:100000002AEF3CF0F76A140FF66E000EF722090093
:10001000F55012000A4E494320696E6974206572DA
:1000200072200000F76A340FF66E000EF722090006
:10003000F5501200204E494320706B742065727297
:100040002000F76A520FF66E000EF7220900F550F5
:100050001200204E49432070747220657272200095
:10006000F76A700FF66E000EF7220900F5501200C5
:100070004E6F2064617974696D650D0A0000F76A3E
:100080008E0FF66E000EF7220900F55012000D0AD1
:1000900053657269616C206E756D3F200000F76AD0
:1000A000AE0FF66E000EF7220900F550120048540C
:1000B00054502F20323030204F4B0D0A0D0A4E6F16
:1000C00020576562207061676573210D0A00F76A29
:1000D000DE0FF66E000EF7220900F550120063687D
:1000E00065636B656400F76AF60FF66E000EF72223
:1000F0000900F550120070617373776F72642E6897
:10010000746D0000F76A140FF66E010EF7220900F5
:10011000F55012006572726F722E68746D00F76A86
:100120002E0FF66E010EF7220900F550120020285E
:10013000444843502900F76A460FF66E010EF72235
:100140000900F55012002028537461746963290076
:10015000F76A600FF66E010EF7220900F5501200E3
:1001600057656220536D61727420503138413639C1
:1001700039390000F76A840FF66E010EF722090084
:10018000F550120056657220312E30360000F76AA5
:100190009E0FF66E010EF7220900F55012004B5328
:1001A0002D313137464D2D560000F76ABA0FF66EE5
:1001B000010EF7220900F55012004B532D31313555
:1001C000464D2D560000F76AD60FF66E010EF72247
:1001D0000900F55012004B5449204E6574776F7238
:1001E0006B730000F76AF40FF66E010EF722090038
:1001F000F55012000D0A44484350204950207363C3
:10020000616E6E696E670000F76A180FF66E020E77
:10021000F7220900F55012004B533131372D000001
:10022000F76A300FF66E020EF7220900F550120041
:100230004B533131352D0000F76A480FF66E020E30
:10024000F7220900F55012000D0A0D0A0000F76AA6
:100250005E0FF66E020EF7220900F5501200576588
:100260006220536D61727420503138413600F76A54
:100270007E0FF66E020EF7220900F5501200436F52
:100280006E6669672000F76A960FF66E020EF72217
:100290000900F55012000D0A0D0A495020616464EE
:1002A000723A2000F76AB40FF66E020EF7220900C8
:1002B000F55012000D0A4E65746D61736B3A2000A3
:1002C000F76AD00FF66E020EF7220900F550120001
:1002D0000D0A476174657761792049503A20000022
:1002E000F76AF00FF66E020EF7220900F5501200C1
:1002F0000D0A4D616320616464723A200000F76A60
:100300000E0FF66E030EF7220900F55012000D0ACB
:10031000393343343620436865636B00F76A2C0F2A
:10032000F66E030EF7220900F5501200204F4B2005
:100330002100F76A420FF66E030EF7220900F5500E
:100340001200204661696C6564202100F76A5C0F29
:10035000F66E030EF7220900F55012000D0A5254F2
:100360004C3830313920436865636B00F76A7C0F85
:10037000F66E030EF7220900F55012000D0A323412
:100380004C4332353620436865636B00010EEA6EDC
:10039000640EE96EEF50D8B4DBEF01F0060E016E8B
:1003A000006A002EFED7012EFBD77B0E006E002EBA
:1003B000FED7EF2EF3D7000C01011A51E96E1B5145
:1003C000EA6E00011FC1EFFF010E01011A25E96E5F
:1003D000000E1B21EA6E00011EC1EFFF020E01019B
:1003E0001A25E96E000E1B21EA6E00011DC1EFFF08
:1003F000030E01011A25E96E000E1B21EA6E0001B1
:100400001CC1EFFF000C0101636B626B0001010175
:1004100062510508D8B003D000011EEF02F00001C0
:1004200062C1A9FFA69CA69EA680A85001016327D1
:1004300000010101622B000107EF02F00101631FBF
:100440006351016E0001000CA96A36C0A8FFA69C8A
:10045000A69EA684F250006EF29E0F01550EA76E66
:10046000AA0EA76EA6820001A6B234EF02F0A694EF
:100470000050F212010EA96E37C0A8FFA69CA69EDE
:10048000A684F250006EF29E0F01550EA76EAA0EC2
:10049000A76EA6820001A6B24BEF02F0A694005010
:1004A000F212020EA96E1CC0A8FFA69CA69EA684EE
:1004B000F250006EF29E0F01550EA76EAA0EA76EA7
:1004C000A6820001A6B262EF02F0A6940050F212DA
:1004D000030EA96E1BC0A8FFA69CA69EA684F25080
:1004E000006EF29E0F01550EA76EAA0EA76EA68291
:1004F0000001A6B279EF02F0A6940050F212040EA9
:10050000A96E1AC0A8FFA69CA69EA684F250006EF3
:10051000F29E0F01550EA76EAA0EA76EA6820001CD
:10052000A6B290EF02F0A6940050F212050EA96E4A
:1005300019C0A8FFA69CA69EA684F250006EF29E4B
:100540000F01550EA76EAA0EA76EA6820001A6B2D5
:10055000A7EF02F0A6940050F212130EA96E24C069
:10056000A8FFA69CA69EA684F250006EF29E0F01E4
:10057000550EA76EAA0EA76EA6820001A6B2BEEF08
:1005800002F0A6940050F212140EA96E23C0A8FF28
:10059000A69CA69EA684F250006EF29E0F01550EF8
:1005A000A76EAA0EA76EA6820001A6B2D5EF02F032
:1005B000A6940050F212150EA96E22C0A8FFA69CA8
:1005C000A69EA684F250006EF29E0F01550EA76EF5
:1005D000AA0EA76EA6820001A6B2ECEF02F0A694C6
:1005E0000050F212160EA96E21C0A8FFA69CA69E6E
:1005F000A684F250006EF29E0F01550EA76EAA0E51
:10060000A76EA6820001A6B203EF03F0A6940050E5
:10061000F212170EA96E28C0A8FFA69CA69EA6845B
:10062000F250006EF29E0F01550EA76EAA0EA76E35
:10063000A6820001A6B21AEF03F0A6940050F212AF
:10064000180EA96E27C0A8FFA69CA69EA684F250ED
:10065000006EF29E0F01550EA76EAA0EA76EA6821F
:100660000001A6B231EF03F0A6940050F212190E69
:10067000A96E26C0A8FFA69CA69EA684F250006E76
:10068000F29E0F01550EA76EAA0EA76EA68200015C
:10069000A6B248EF03F0A6940050F2121A0EA96E0B
:1006A00025C0A8FFA69CA69EA684F250006EF29ECE
:1006B0000F01550EA76EAA0EA76EA6820001A6B264
:1006C0005FEF03F0A6940050F21203EC02F001C0B9
:1006D0001AF1060EA96E1AC1A8FFA69CA69EA684B2
:1006E000F250006EF29E0F01550EA76EAA0EA76E75
:1006F000A6820001A6B27AEF03F0A6940050F2128F
:10070000000C899289948996800E0101566F090E1A
:10071000576F010E586F0001010158510408D8B0FD
:1007200003D000019FEF03F00001D890010156377C
:10073000573700010101582B00018CEF03F0898627
:10074000020E0101646F0001C6EC01F0010E01010F
:10075000586F0001010158510A08D8B003D00001B8
:10076000C8EF03F00001D890010156375737D8A0E1
:1007700003D00001C0EF03F000018992C1EF03F044
:100780008982898489940101582B0001AAEF03F022
:100790008992020E0101646F0001C6EC01F0899696
:1007A000080E006E002EFED789848994000C01018A
:1007B0005E355F6F5F37FC0E5F175D35646F6437C2
:1007C000FC0E64175E39006E00320032030E001614
:1007D00000506411606F5C35646F6437FC0E641701
:1007E0005D39006E00320032030E001600506411B5
:1007F000616F050E626F010E636F000101016351AD
:100800000508D8B003D0000113EF04F00001D89020
:1008100001015F3760376137623700010101632BE7
:100820000001FEEF03F08986020E0101646F0001F2
:10083000C6EC01F08980010E0101636F0001010126
:1008400063511908D8B003D000013FEF04F0000154
:10085000D89001015F37603761376237D8A003D085
:10086000000137EF04F00001899238EF04F089822B
:10087000898489940101632B00011FEF04F08992A0
:100880008996030E006E002EFED789848994030E8C
:10089000006E002EFED7898689848994000E80B070
:1008A000010E0108D8B44CEF04F0020E0101646F90
:1008B0000001C6EC01F08996080E006E002EFED7EE
:1008C00089848994320E0101646F0001C6EC01F045
:1008D000000C020EA96E56C1A8FFA69CA69EA68477
:1008E000F250006EF29E0F01550EA76EAA0EA76E73
:1008F000A6820001A6B27AEF04F0A6940050F2128C
:10090000030EA96E57C1A8FFA69CA69EA684F2500E
:10091000006EF29E0F01550EA76EAA0EA76EA6825C
:100920000001A6B291EF04F0A6940050F212040E5A
:10093000A96E58C1A8FFA69CA69EA684F250006E80
:10094000F29E0F01550EA76EAA0EA76EA682000199
:10095000A6B2A8EF04F0A6940050F212050EA96EFC
:1009600059C1A8FFA69CA69EA684F250006EF29ED6
:100970000F01550EA76EAA0EA76EA6820001A6B2A1
:10098000BFEF04F0A6940050F21203EC02F001C095
:1009900062F1060EA96E62C1A8FFA69CA69EA6845F
:1009A000F250006EF29E0F01550EA76EAA0EA76EB2
:1009B000A6820001A6B2DAEF04F0A6940050F2126B
:1009C000130EA96E5AC1A8FFA69CA69EA684F2503B
:1009D000006EF29E0F01550EA76EAA0EA76EA6829C
:1009E0000001A6B2F1EF04F0A6940050F212140E2A
:1009F000A96E5BC1A8FFA69CA69EA684F250006EBD
:100A0000F29E0F01550EA76EAA0EA76EA6820001D8
:100A1000A6B208EF05F0A6940050F212150EA96ECA
:100A20005CC1A8FFA69CA69EA684F250006EF29E12
:100A30000F01550EA76EAA0EA76EA6820001A6B2E0
:100A40001FEF05F0A6940050F212160EA96E5DC1BC
:100A5000A8FFA69CA69EA684F250006EF29E0F01EF
:100A6000550EA76EAA0EA76EA6820001A6B236EF9B
:100A700005F0A6940050F212170EA96E5EC1A8FFF1
:100A8000A69CA69EA684F250006EF29E0F01550E03
:100A9000A76EAA0EA76EA6820001A6B24DEF05F0C2
:100AA000A6940050F212180EA96E5FC1A8FFA69C72
:100AB000A69EA684F250006EF29E0F01550EA76E00
:100AC000AA0EA76EA6820001A6B264EF05F0A69456
:100AD0000050F212190EA96E60C1A8FFA69CA69E36
:100AE000A684F250006EF29E0F01550EA76EAA0E5C
:100AF000A76EA6820001A6B27BEF05F0A694005077
:100B0000F2121A0EA96E61C1A8FFA69CA69EA68429
:100B1000F250006EF29E0F01550EA76EAA0EA76E40
:100B2000A6820001A6B292EF05F0A6940050F21240
:100B300035EF07F0010E926E81EC03F001015C6B62
:100B4000410E5D6F540E5E6F0001D7EC03F0130E83
:100B50000101556F0001010155512208D8B003D0A1
:100B60000001C3EF05F0000155C15CF1FF0E01016A
:100B70005D6F040E5E6F0001D7EC03F00101552B91
:100B80000001ABEF05F0140E01015C6FFF0E5D6F0D
:100B9000FF0E5E6F0001D7EC03F0230E0101556FCD
:100BA0000001010155513F08D8B003D00001E7EF23
:100BB00005F0000155C15CF101015D6B5E6B000148
:100BC000D7EC03F00101552B0001D1EF05F0010E28
:100BD0000101556F0001010155510908D8B003D03A
:100BE000000103EF06F0000155C15CF1840E010124
:100BF0005D6F4F0E5E6F0001D7EC03F00101552BC6
:100C00000001EBEF05F0030E01015C6F840E5D6FD8
:100C1000410E5E6F0001D7EC03F0080E01015C6F1E
:100C2000C40E5D6F4D0E5E6F0001D7EC03F00A0E2F
:100C300001015C6F590E5D6F020E5E6F0001D7EC13
:100C400003F00B0E01015C6F800E5D6F5E6B0001A7
:100C5000D7EC03F00C0E01015C6FFA0E5D6F500EC5
:100C60005E6F0001D7EC03F00D0E01015C6FFA0E10
:100C70005D6F500E5E6F0001D7EC03F00E0E0101A8
:100C80005C6F550E5D6F5E6B0001D7EC03F00F0ECD
:100C900001015C6F550E5D6F5E6B0001D7EC03F0D8
:100CA000100E01015C6F300E5D6F5E6B0001D7ECC2
:100CB00003F0110E01015C6FFF0E5D6F5E6B0001B2
:100CC000D7EC03F0120E01015C6F360E5D6F5E6BA8
:100CD0000001D7EC03F02C0E01015C6FD00E5D6FAC
:100CE0005E6B0001D7EC03F02D0E01015C6F450E29
:100CF0005D6F560E5E6F0001D7EC03F00101556B7E
:100D00000001010155510708D8B003D00001AAEF36
:100D100006F000010A0E01015525566F000156C16B
:100D2000A9FFA86AA69CA69EA684F250006EF29E19
:100D30000F01550EA76EAA0EA76EA6820001A6B2DD
:100D40009FEF06F0A6940050F2120101552B00010E
:100D500081EF06F00A0EA96E310EA86EA69CA69E23
:100D6000A684F250006EF29E0F01550EA76EAA0ED9
:100D7000A76EA6820001A6B2BBEF06F0A6940050B3
:100D8000F2120B0EA96E320EA86EA69CA69EA68429
:100D9000F250006EF29E0F01550EA76EAA0EA76EBE
:100DA000A6820001A6B2D2EF06F0A6940050F2127D
:100DB0000C0EA96E330EA86EA69CA69EA684F250B9
:100DC000006EF29E0F01550EA76EAA0EA76EA682A8
:100DD0000001A6B2E9EF06F0A6940050F212080E48
:100DE000A96EA86AA69CA69EA684F250006EF29EEA
:100DF0000F01550EA76EAA0EA76EA6820001A6B21D
:100E0000FFEF06F0A6940050F212090EA96E020E32
:100E1000A86EA69CA69EA684F250006EF29E0F01BC
:100E2000550EA76EAA0EA76EA6820001A6B216EFF7
:100E300007F0A6940050F212C00E0101566FA80EE2
:100E4000576F586B020E596FFF0E5A6FFF0E5B6F94
:100E5000FF0E5C6F5D6BC00E5E6FA80E5F6F606B08
:100E6000010E616F000169EF04F0000C21C103F075
:100E700001012051E96E000103C0EAFFECCF03F04D
:100E8000ED52EF50105C0101246F03501158256F93
:100E900022512311D8A403D0000165EF07F000010F
:100EA00001012351255DD8B003D0000176EF07F092
:100EB0000001D8A465EF07F001012251245DD8B0EC
:100EC00003D0000176EF07F0000121C103F001011A
:100ED0002051E96E000103C0EAFF11C0ECFFED52A2
:100EE00010C0EFFF010E016E78EF07F0000E016EEB
:100EF000000C74C181FF75C183FF000E956E849252
:100F000000008482FF0E956E000C0E0E0101712709
:100F1000400E7223070E746F400E756F000179EC5E
:100F200007F0080E0101746F000171C175F179ECD1
:100F300007F072C173F1090E0101746F000173C1F2
:100F400075F179EC07F0010E6C6E000CFF0E956EDA
:100F500071C181FF849083CF72F18480010172514D
:100F6000016E0001000C01016F6B000171C070F196
:100F700001017053D8B403D00001C2EF07F00001A3
:100F800020EF08F001017051010B7027070E746FFC
:100F9000400E756F000179EC07F00A0E0101746FC5
:100FA000000170C175F179EC07F00B0E0101746F4F
:100FB000756B000179EC07F00101746B120E756F0F
:100FC000000179EC07F0100E816E000E956E0101A4
:100FD00070517007000AD8A403D0000101EF08F097
:100FE000000101016F516F2B720FE96EEA6AD8B0F0
:100FF000EA2AEF50836E8492000084820001E7EFBA
:1010000007F0FF0E956EFF0E0101706F00010101E8
:101010007053D8A403D0000120EF08F00001070EA0
:101020000101716F0001A6EC07F00150400B000AAE
:10103000D8A420EF08F001017007000107EF08F0C5
:10104000000C7152D8B43AEF08F06C52D8A437EFC4
:1010500008F071506F5C01016F6F000E7058706F77
:10106000000170C172F16FC171F185EC07F0B3EC52
:1010700007F0716A6E50705CD8A04BEF08F0D8A4EE
:1010800047EF08F06F506D5CD8B04BEF08F070C0C0
:101090006EF06FC06DF0000C29A061EF08F0010147
:1010A0006F512B266F512B5CD8A003D000015FEF4E
:1010B00008F000012A2AD8A45FEF08F02B2A71EF6C
:1010C00008F001016F512A266F512A5CD8A003D085
:1010D000000171EF08F000012B2AD8A471EF08F08D
:1010E0002A2A2970000C70500408D8B085EF08F047
:1010F000FF0AD8A481EF08F06F50E908D8B085EF57
:1011000008F0000E016E9EEF08F071501F08D8B075
:101110008CEF08F021EC08F07150712A720FE96E23
:10112000EA6AD8B0EA2A6EC1EFFF6F2AD8B4702AF3
:101130006EC16FF14CEC08F0010E016E000C29A697
:10114000B7EF08F001016D510A08D8B403D00001CF
:10115000B0EF08F000010D0E9EA8ACEF08F0AD6EE8
:1011600001016D5100019EA8B3EF08F0AD6E29A8F2
:10117000BEEF08F06DC16EF173EC08F0000CA96AC7
:10118000A69CA69EA680A850366E010EA96EA69CAF
:10119000A69EA680A850376E020EA96EA69CA69E9B
:1011A000A680A8501C6E030EA96EA69CA69EA680C3
:1011B000A8501B6E040EA96EA69CA69EA680A850E1
:1011C0001A6E050EA96EA69CA69EA680A850196E42
:1011D000130EA96EA69CA69EA680A850246E140E7F
:1011E000A96EA69CA69EA680A850236E150EA96E79
:1011F000A69CA69EA680A850226E160EA96EA69C3E
:10120000A69EA680A850216E170EA96EA69CA69E2B
:10121000A680A850286E180EA96EA69CA69EA68031
:10122000A850276E190EA96EA69CA69EA680A8504F
:10123000266E1A0EA96EA69CA69EA680A850256EA4
:10124000060EA96EA69CA69EA680A8500101186F46
:10125000000103EC02F001011851015CD8A403D095
:10126000000137EF09F00001000E38EF09F0010E20
:10127000016E000C3A50010170273B5071237151EF
:101280005E08D8A003D0000152EF09F0000101016F
:101290007051016EE70E7125036E0150706F0001F1
:1012A00003C071F1070E0101746F400E756F0001EC
:1012B00079EC07F0080E0101746F000170C175F13F
:1012C00079EC07F071C172F1090E0101746F000130
:1012D00072C175F179EC07F06C6A000C416A41C08B
:1012E00040F03F6A40C03EF0149C299A0101716BA6
:1012F000706B00013AEC09F0000C9EAA8EEF09F029
:10130000ABB48AEF09F0ABB28AEF09F0010E016EBF
:1013100090EF09F0AB98AECF20F1AB88000E016ED4
:10132000DCEF09F001011651CF5C156F15517908FA
:10133000D8A003D00001A9EF09F00001102AD8B409
:10134000112A7A0E01011627010E016E0001ABEF82
:1013500009F0000E016EB0EF09F0040092EF09F001
:10136000000C9EBACBEF09F0ABB4BAEF09F0ABA218
:10137000CBEF09F0ABB4C0EF09F0ABA2C8EF09F0B6
:10138000AB98AECF20F1AB88000E016ECDEF09F027
:101390000400B1EF09F0AE50016E0CEF0AF001014C
:1013A0001C6B010E216F1D0E206F236B226B000141
:1013B00036EC07F07DEF09F00152D8A40AEF0AF0ED
:1013C00001011A511B11D8A403D0000106EF0AF045
:1013D0000001010E0101216F1D0E206F00011BC1D4
:1013E00023F11AC122F136EC07F00152D8B406EF0E
:1013F0000AF0420E01011C25E96EEA6AD8B0EA2A19
:10140000EF6A1C51016E0001B4EF0AF0ADEC09F077
:10141000DAEF09F0B1EF09F001C01FF101011F512E
:101420001F08D8A003D0000120EF0AF0000101013D
:101430001F517F08D8B403D000017CEF0AF00001EF
:1014400001011F511B08D8B403D0000130EF0AF08E
:10145000000101011C6B0001A2EF0AF07AEF0AF013
:1014600001011F510D08D8B403D000014EEF0AF05E
:10147000000101011A511B11D8A403D000014AEF49
:101480000AF0000101011C53D8A403D000014CEF65
:101490000AF00001A2EF0AF07AEF0AF001011F51F1
:1014A0000808D8A403D0000160EF0AF00001010190
:1014B0001F517F08D8B403D000017AEF0AF0000171
:1014C00001011C53D8A403D000017AEF0AF00001F7
:1014D00001011C07080E00019EA86CEF0AF0AD6E1A
:1014E000200E9EA871EF0AF0AD6E080E9EA876EF52
:1014F0000AF0AD6EA0EF0AF001011C512808D8B027
:1015000003D00001A0EF0AF0000101011C511C2BC7
:10151000420FE96EEA6AD8B0EA2A00011FC1EFFF64
:1015200001011A511B11D8B403D00001A0EF0AF039
:10153000000101011F5100019EA89CEF0AF0AD6E51
:10154000DAEF09F0420E01011C25E96EEA6AD8B013
:10155000EA2AEF6A3D6A00011CC13CF03CC040F041
:1015600001011C51016E0001B6EF0CF00101705336
:10157000D8B403D00001C0EF0AF00001F9EF0AF07F
:10158000070E0101746F400E756F000179EC07F0D2
:101590000A0E0101746F000170C175F179EC07F05A
:1015A0000B0E0101746F756B000179EC07F00101FE
:1015B000746B0A0E756F000179EC07F0100E816EE6
:1015C000FF0E956E010170517007000AD8A403D078
:1015D0000001F9EF0AF0000184904050402A420FC8
:1015E000E96EEA6AD8B0EA2A83CFEFFF8480E2EF9F
:1015F0000AF0000C415001016A5DD8A003D000013F
:101600002EEF0BF000016AC16CF14050415CD8B084
:101610002AEF0BF001016C516C2B420F016E036A33
:10162000D8B0032A0150716F000103C072F141501C
:10163000412A420FE96EEA6AD8B0EA2AEF50010166
:10164000746F000172C1EAFF71C1E9FF74C1EFFF5D
:1016500005EF0BF06CC140F06AC141F03E503C5CBC
:1016600001016E6F3F503D586F6F6F53D8B403D078
:1016700000014CEF0BF0000101016B516E5DD8A031
:1016800003D000014CEF0BF000016FC103F001012A
:101690006E5100014FEF0BF001016B510001010190
:1016A0006B6F2A0ED88040546B5DD8A403D0000124
:1016B00065EF0BF0D8B003D0000165EF0BF000012F
:1016C0002A0ED880405468EF0BF001016B510001E5
:1016D00001016B6F00016BC16DF101016D53D8A465
:1016E00003D0000183EF0BF000016C52D8B47FEF00
:1016F0000BF03FC071F13EC070F13AEC09F06BC1E4
:1017000070F1B6EC0AF001016B51016E0001000CA2
:101710004050415CD8A095EF0BF00A0E01016A6FB2
:101720002A0E6B6F0001FAEC0AF04050415CD8A021
:101730009EEF0BF0000E016EC1EF0BF04150412AFD
:10174000420FE96EEA6AD8B0EA2AEF500101696FE8
:101750003E2AD8B43F2A29AA03D00001B5EF0BF0E6
:10176000000169C16FF14CEC08F068C103F00101A0
:101770006751E96E000103C0EAFF69C1EFFF010E86
:10178000016E000C4152D8B4DCEF0BF03E503F101C
:10179000D8B4DCEF0BF04106420E4124E96EEA6A50
:1017A000D8B0EA2A20C1EFFF3E50D8B43F063E062B
:1017B000010E016EDEEF0BF0000E016E76EF0CF005
:1017C00001011C6B1D6B1F6B0001010E0101686F95
:1017D0001E0E676F000188EC0BF00152D8B47AEF4F
:1017E0000CF001011E512F08D8A003D000011CEFFE
:1017F0000CF0000101011E513908D8B003D00001DE
:101800001CEF0CF0000101011F2B300E1E5F1C3578
:10181000206F1D35216F20372137203721372037A2
:101820002137F00E20171E5120251C6F000E21219C
:101830001D6F000178EF0CF001011E514008D8A087
:1018400003D0000147EF0CF0000101011E514608D2
:10185000D8B003D0000147EF0CF0000101011F2BAD
:10186000370E1E5F1C35206F1D35216F2037213745
:101870002037213720372137F00E20171E51202521
:101880001C6F000E21211D6F000178EF0CF001018B
:101890001E516008D8A003D0000172EF0CF00001C7
:1018A00001011E516608D8B003D0000172EF0CF0A0
:1018B000000101011F2B570E1E5F1C35206F1D35C7
:1018C000216F203721372037213720372137F00E7D
:1018D00020171E5120251C6F000E21211D6F0001B5
:1018E00078EF0CF01EC120F1C2EF0BF07AEF0CF094
:1018F000E5EF0BF01BC103F001011A51E96E000185
:1019000003C0EAFF1DC1ECFFED521CC1EFFF010156
:101910001F53D8B403D0000192EF0CF00001000E69
:1019200093EF0CF0010E016EC2EF0CF001011A6B87
:10193000000101011A5100013FEC00F001011A2BD6
:1019400000019EA8A1EF0CF0AD6E0E0E01011A5D14
:10195000D8B403D0000199EF0CF000016EEC09F04F
:1019600001011B6B1A6B0001CFEF09F00152D8B4D3
:10197000CAEF0CF0010E01011B6F180E1A6F000167
:10198000E0EF0BF00152D8B4CAEF0CF019C136F0F9
:1019900018C137F00D0E9EA8CBEF0CF0AD6E0A0EFD
:1019A0009EA8D0EF0CF0AD6E01011B6B190E1A6FE3
:1019B000C00E1C6FA80E1D6F1E6B020E1F6F000164
:1019C000DCEC01F001011B6B210E1A6FFF0E1C6F86
:1019D000FF0E1D6FFF0E1E6F1F6B0001DCEC01F090
:1019E00001011B6B250E1A6FC00E1C6FA80E1D6F18
:1019F0001E6B010E1F6F0001DCEC01F024EC02F005
:101A0000010E016ED6EF3DF0D89001015535566FAD
:101A1000B40E576F000E926E8996010E586F00013A
:101A2000010158512008D8B003D0000121EF0DF07A
:101A300000018982899489840101582B000110EFEB
:101A40000DF0010E0101586F0001010158512F08DE
:101A5000D8B003D0000171EF0DF000010101585121
:101A60000F08D8B003D0000145EF0DF00001D89069
:101A7000010156375737D8A003D0000144EF0DF0CD
:101A80000001899245EF0DF0898289940101585136
:101A90000F08D8A003D000015CEF0DF0000180B268
:101AA00055EF0DF0D89056EF0DF0D88001015B375F
:101AB0005C375D375E3700018984010158510F089A
:101AC000D8B403D000016CEF0DF00001020E926E4D
:101AD00089948984899489840101582B000125EF18
:101AE0000DF05BC100F05CC101F05DC102F05EC1B0
:101AF00003F0000C010120AF03D0000199EF0DF0BD
:101B00000F0E006E1F3900160A0E005CD8A003D01D
:101B1000000190EF0DF0300E0026000194EF0DF063
:101B2000010120510026000100509EA895EF0DF004
:101B3000AD6E0F0E01011F170A0E1F5DD8A003D056
:101B40000001A7EF0DF0300E0001ABEF0DF0010129
:101B5000209F2051000101011F271F5100019EA855
:101B6000AFEF0DF0AD6E000C0101586B596B57359E
:101B70005A6F5A37FC0E5A17060E5B6F010E5C6FD8
:101B8000000101015C510508D8B003D00001D6EF77
:101B90000DF00001D8900101583759375A375B379B
:101BA000000101015C2B0001C1EF0DF08986010EDF
:101BB00001015C6F000101015C511908D8B003D02C
:101BC00000010FEF0EF00001D8900101583759378E
:101BD0005A375B37D8A003D00001F3EF0DF00001B6
:101BE0008992F4EF0DF089828984899401015C5116
:101BF0000908D8A003D000010AEF0EF0000180B060
:101C000005EF0EF0D89006EF0EF0D88001015F3797
:101C10006037000101015C2B0001DBEF0DF08996BC
:101C200001015F51016E6051026E0001000C080E4F
:101C3000016E000004008B96949604000101643745
:101C40008298D8B09488D8A094989486000182A6EF
:101C500027EF0EF0012E19EF0EF004008B969496EC
:101C60000000948804000400948682A635EF0EF0EC
:101C7000016A040082B801808B96949682989498A9
:101C8000000C080E0101686F000100C069F1948822
:101C90000400948682A64AEF0EF082B8D88082A80B
:101CA000D8900136040094968B960101682F02D0DB
:101CB00004D00001000147EF0EF0948804008298E0
:101CC0006951D8A4949800010000948682A666EF1A
:101CD0000EF004008B969496040082989498000C61
:101CE000010E0101556F0001E76B94880400948692
:101CF00004008298949804008B969496A00E01019B
:101D0000646F000117EC0EF00101646B000117EC29
:101D10000EF00101646B000117EC0EF094980000C6
:101D2000948682A691EF0EF00400000000000000EF
:101D300094880400948804009486040082989498FF
:101D400004008B969496A10E0101646F000117ECBC
:101D50000EF00101566B0001010156510608D8B082
:101D600003D00001C8EF0EF00001D40E010156258A
:101D7000E96EEA6AD8B0EA2A010E006E000141EC71
:101D80000EF00150EF6E0101562B0001ACEF0EF08A
:101D9000D43DD5EF0EF0D53DD5EF0EF0006A41EC05
:101DA0000EF040EF0FF026EF0FF00101556B566B70
:101DB0000001010156510B08D8B003D000011FEFFC
:101DC0000FF00001580E01015625E96E010EEA6E72
:101DD000D8B0EA2A56510A08D8A003D00001F5EF7E
:101DE0000EF00001000EF6EF0EF0010E0101666F1D
:101DF000000166C100F041EC0EF001C057F157C17F
:101E0000EFFF070E01015625016E036AD8B0032AC1
:101E10000150D40FE96E000E0320EA6EEF50575DBB
:101E2000D8A403D000011AEF0FF00001010E010148
:101E3000556F00010101562B0001D9EF0EF0DB5365
:101E4000D8A426EF0FF00101556B00019498000013
:101E5000948682A629EF0FF0040000000000000025
:101E600094880400E72BE7516308D8A040EF0FF0F7
:101E700001015553D8B403D000019AEF0EF00001D0
:101E800001015553D8A403D000014AEF0FF000011F
:101E9000D56BD46B01015553D8A403D0000155EF85
:101EA0000FF00001000E56EF0FF0010E016E000C56
:101EB0000101556B000104EC0DF003C01BF102C0E1
:101EC0001AF101C019F100C018F1300E9EA866EF9A
:101ED0000FF0AD6E780E9EA86BEF0FF0AD6E1BC1CC
:101EE0001FF1370E0101206F00017AEC0DF01AC1CD
:101EF0001FF1370E0101206F00017AEC0DF019C1BE
:101F00001FF1370E0101206F00017AEC0DF018C1AE
:101F10001FF1370E0101206F00017AEC0DF0200E49
:101F20009EA890EF0FF0AD6E0101186B000101014A
:101F3000185100017FEC01F00101182B00019EA84F
:101F40009FEF0FF0AD6E0D0E0101185DD8B403D0F8
:101F5000000197EF0FF0090E196F00012E0E9EA8D9
:101F6000AFEF0FF0AD6E0101192F02D004D00001C8
:101F70000001AEEF0FF0010E926E000181EC03F054
:101F80000101576B0001B4EC0DF002C019F101C062
:101F900018F1010118515408D8B403D00001F5EF2D
:101FA0000FF00001010119514108D8B403D000011C
:101FB000F5EF0FF000010101186B0001010118514C
:101FC00000018EEC01F00101182B00019EA8E6EF44
:101FD0000FF0AD6E050E0101185DD8B403D00001FD
:101FE000DEEF0FF000010DEF10F00101186B0001A2
:101FF00001011851000199EC01F00101182B0001B9
:102000009EA800EF10F0AD6E090E0101185DD8B466
:1020100003D00001F8EF0FF000010101186B00017F
:10202000010118510001A6EC01F00101182B00017B
:102030009EA818EF10F0AD6E0F0E0101185DD8B418
:1020400003D0000110EF10F0070E196F00012E0EE3
:102050009EA828EF10F0AD6E0101192F02D004D018
:102060000001000127EF10F0070E716F0001A6ECD0
:1020700007F00150800B000AD8A459EF10F00101BD
:10208000186B000101011851000199EC01F00101E8
:10209000182B00019EA84AEF10F0AD6E090E010149
:1020A000185DD8B403D0000142EF10F0000171EFC9
:1020B00010F00101186B00010101185100018EECB4
:1020C00001F00101182B00019EA864EF10F0AD6E25
:1020D000050E0101185DD8B403D000015CEF10F0CB
:1020E00000010101186B0001010118510001B6EC5B
:1020F00001F00101182B00019EA87CEF10F0AD6EDD
:102100000F0E0101185DD8B403D0000174EF10F078
:10211000070E196F00012E0E9EA88CEF10F0AD6E09
:102120000101192F02D004D0000100018BEF10F043
:10213000000170EC0EF0E753D8A4B9EF10F00101E4
:10214000186B000101011851000199EC01F0010127
:10215000182B00019EA8AAEF10F0AD6E090E010128
:10216000185DD8B403D00001A2EF10F00001D1EF48
:1021700010F00101186B00010101185100018EECF3
:1021800001F00101182B00019EA8C4EF10F0AD6E04
:10219000050E0101185DD8B403D00001BCEF10F0AA
:1021A000000137EF3EF0FF0E956E816AF19E200E22
:1021B000936E848084828484969096929694E3EFC2
:1021C00010F0D3EF10F0020E0101646F0001C6ECB5
:1021D00001F08494020E0101646F0001C6EC01F06D
:1021E0001F0E0101716F0001A6EC07F001C01CF188
:1021F0001F0E0101746F00011CC175F179EC07F02D
:10220000020E0101646F0001C6EC01F0070E01012E
:10221000716F0001A6EC07F00150800B000AD8A4F2
:102220002EEF11F001011C6B000101011C51000196
:1022300002EC00F001011C2B00019EA81DEF11F023
:10224000AD6E0E0E01011C5DD8B403D0000115EF78
:1022500011F0000E016E000110EF12F00101746B1D
:10226000210E756F000179EC07F0020E0101646F19
:102270000001C6EC01F00E0E0101746F480E756F7F
:10228000000179EC07F00A0E0101746F756B000113
:1022900079EC07F00B0E0101746F756B000179EC9E
:1022A00007F00C0E0101746F200E756F000179ECC0
:1022B00007F00D0E0101746F020E756F000179ECCD
:1022C00007F0040E0101746F400E756F000179EC88
:1022D00007F0010E0101746F460E756F000179EC75
:1022E00007F0020E0101746F5F0E756F000179EC4B
:1022F00007F0030E0101746F5E0E756F000179EC3B
:1023000007F0070E0101746FFF0E756F000179EC85
:1023100007F00F0E0101746F756B000179EC07F087
:102320000101746B610E756F000179EC07F0020E0C
:102330000101646F0001C6EC01F001011B6B00019B
:1023400001011B510508D8B003D00001C1EF11F005
:102350000001010E01011B251C6F320E1B25E96EC9
:10236000EA6AD8B0EA2A0001EFCF1DF11CC174F16E
:102370001DC175F179EC07F001011B2B0001A0EFE5
:1023800011F001011B6B000101011B510708D8B0BE
:1023900003D00001DFEF11F00001080E01011B2541
:1023A0001C6F00011CC174F1FF0E0101756F00016B
:1023B00079EC07F001011B2B0001C4EF11F0070EAF
:1023C0000101746F470E756F000179EC07F0470E3D
:1023D000386E0101746B200E756F000179EC07F007
:1023E0000C0E0101746F040E756F000179EC07F09B
:1023F0000D0E0101746F756B000179EC07F0070E8B
:102400000101746FFF0E756F000179EC07F0010197
:10241000746B220E756F000179EC07F0010E016EEE
:10242000000C016A026A006A036A01017251D8B4A1
:1024300003D0000123EF12F07151D8A403D00001A2
:102440004EEF12F00001100E0101736F0001D890E1
:1024500001016F377037003603367251035CD8B410
:1024600003D0000137EF12F07151005C0001D8A0D9
:1024700043EF12F001017151005ED8A003067251C2
:10248000035ED8800001013602360101732F02D0AD
:1024900004D00001000127EF12F000010000000C41
:1024A0000101666B000101016651662B670FE96E41
:1024B000010EEA6ED8B0EA2A000164C170F163C16E
:1024C0006FF10101726B0A0E716F000111EC12F0D5
:1024D0000050300FEF6E64C170F163C16FF1010104
:1024E000726B0A0E716F000111EC12F002C064F100
:1024F00001C063F1010163516411D8B403D000013C
:1025000053EF12F0000166C165F101016653D8A4D2
:1025100003D000019FEF12F0000101016607670E72
:102520006625E96E010EEA6ED8B0EA2A0001EFCF07
:102530006CF16CC16DF19FEC08F085EF12F00101B8
:102540006551016E0001000C29862984299801013A
:102550001D6B000101011D51000143EC01F001015F
:102560001D2B00019EA8B2EF12F0AD6E0D0E010101
:102570001D5DD8B403D00001AAEF12F0646B000116
:102580001CC063F150EC12F02E0E01016D6F0001C2
:102590009FEC08F00101646B00011BC063F150EC7B
:1025A00012F02E0E01016D6F00019FEC08F0010189
:1025B000646B00011AC063F150EC12F02E0E0101A1
:1025C0006D6F00019FEC08F00101646B000119C000
:1025D00063F150EC12F0000C29862984299801013E
:1025E0001D6B000101011D51000152EC01F00101C0
:1025F0001D2B00019EA8FAEF12F0AD6E0B0E01012B
:102600001D5DD8B403D00001F2EF12F0646B00013D
:1026100024C063F150EC12F02E0E01016D6F000129
:102620009FEC08F00101646B000123C063F150ECE2
:1026300012F02E0E01016D6F00019FEC08F00101F8
:10264000646B000122C063F150EC12F02E0E010108
:102650006D6F00019FEC08F00101646B000121C067
:1026600063F150EC12F0000C2986298429980101AD
:102670001D6B000101011D51000160EC01F0010121
:102680001D2B00019EA842EF13F0AD6E0E0E01014E
:102690001D5DD8B403D000013AEF13F0646B000164
:1026A00028C063F150EC12F02E0E01016D6F000195
:1026B0009FEC08F00101646B000127C063F150EC4E
:1026C00012F02E0E01016D6F00019FEC08F0010168
:1026D000646B000126C063F150EC12F02E0E010174
:1026E0006D6F00019FEC08F00101646B000125C0D3
:1026F00063F150EC12F0000C01011E6B00010101AE
:102700001E51000170EC01F001011E2B00019EA87A
:1027100087EF13F0AD6E0C0E01011E5DD8B403D02F
:1027200000017FEF13F01D6B000101011D51040832
:10273000D8B003D00001BAEF13F00001320E01014E
:102740001D25E96EEA6AD8B0EA2A0001EFCF1EF132
:102750001EC11FF1370E0101206F00017AEC0DF050
:102760003A0E9EA8B1EF13F0AD6E01011D2B0001D2
:1027700095EF13F037C01FF1370E0101206F0001F4
:102780007AEC0DF0200E9EA8C3EF13F0AD6E000C96
:1027900021C124F10101256B000120C103F0000ECD
:1027A00001012411226F03502511236F2251016E64
:1027B0002351026E0001000C01011F6B1D51000B23
:1027C000006E1E51800B036E00500310D8A403D07E
:1027D0000001FBEF13F0000101011F53D8A403D047
:1027E0000001F7EF13F00001000EF8EF13F0010EF7
:1027F00001011F6F000101011D51000B006E1E51F0
:10280000400B036E00500310D8A403D0000119EF51
:1028100014F0000101011F53D8A403D0000115EFEB
:1028200014F00001000E16EF14F0010E01011F6FED
:10283000000101011D51000B006E1E51100B036EB3
:1028400000500310D8A403D0000137EF14F00001AA
:1028500001011F53D8A403D0000133EF14F000018D
:10286000000E34EF14F0010E01011F6F0001010191
:102870001D51080B006E1E51000B036E005003101B
:10288000D8A403D0000155EF14F0000101011F533B
:10289000D8A403D0000151EF14F00001000E52EF54
:1028A00014F0010E01011F6F000101011D511D25D2
:1028B000206F1E511E21216F1F512025016E000E19
:1028C0002121036E0350026E000179EF14F0010123
:1028D0001C6B000101011C510708D8B003D0000196
:1028E00082EF14F000011BC11EF11AC11DF1DCEFD3
:1028F00013F002C01BF101C01AF101011C2B0001F1
:102900006AEF14F001011A51016E1B51026E0001B1
:102910009BEF18F0010121510408D8A003D0000159
:10292000A4EF14F00001FF0AD8A4A0EF14F00101F5
:102930002051DC08D8A003D00001A4EF14F000015E
:10294000000E016EB2EF14F021EC08F021C170F01E
:1029500020C16FF070C072F16FC071F185EC07F0AB
:10296000010E016E000C030E01012025E96E000E20
:102970002121EA6E0001EFCF22F122C16EF173EC4A
:1029800008F0020E01012025E96E000E2121EA6EF9
:102990000001EFCF22F122C16EF173EC08F0010EBD
:1029A00001012025E96E000E2121EA6E0001EFCF22
:1029B00022F122C16EF173EC08F001012051E96EA1
:1029C0002151EA6E0001EFCF22F122C16EF173ECCA
:1029D00008F0000C01011E511E07000AD8A403D004
:1029E0000001FBEF14F0000101016E6B000173ECBC
:1029F00008F0EAEF14F0000C01012551036E245198
:102A0000D8B4250724070310D8A403D000011DEF74
:102A100015F0000101012351036E2251222BD8B47D
:102A2000232BE96E000103C0EAFFEFCF26F126C198
:102A30006EF173EC08F0FCEF14F0000C21C122F1F0
:102A400022C16EF173EC08F020C16EF173EC08F056
:102A5000000C030E01012025E96E000E2121EA6E13
:102A60000001EFCF22F122C16FF14CEC08F0020E11
:102A700001012025E96E000E2121EA6E0001EFCF51
:102A800022F122C16FF14CEC08F0010E010120256A
:102A9000E96E000E2121EA6E0001EFCF22F122C182
:102AA0006FF14CEC08F001012051E96E2151EA6E02
:102AB0000001EFCF22F122C16FF14CEC08F0000CC5
:102AC0002B6A2BC02AF02990450E01016E6F000180
:102AD00073EC08F001016E6B000173EC08F0C2C0EA
:102AE00021F1C1C020F11EEC15F001016E6B000157
:102AF00073EC08F0C52BC5C06EF173EC08F0010152
:102B0000216B206B00011EEC15F0640E01016E6F4D
:102B1000000173EC08F0AEC06EF173EC08F0010137
:102B2000216B190E206F000129EC15F00101216BBA
:102B3000B30E206F000129EC15F02A500101206F1F
:102B4000201F000120C16EF173EC08F02B50010131
:102B5000206F201F000120C16EF173EC08F001010D
:102B6000216B190E206F0001B3EC14F00101216BF1
:102B7000B30E206F0001B3EC14F0000C22C123F15E
:102B80000101246B000123C16FF14CEC08F021C15D
:102B90006FF14CEC08F0000C2990C3C02AF0C4C0BF
:102BA0002BF0B8C021F1B7C020F11EEC15F0BAC06F
:102BB00021F1B9C020F11EEC15F0E9C021F1E8C007
:102BC00020F11EEC15F00101216B190E206F0001A0
:102BD00029EC15F00101216BB30E206F000129ECE7
:102BE00015F001016F6B00014CEC08F0110E0101B2
:102BF0006F6F00014CEC08F0E9C022F1E8C021F150
:102C0000BEEC15F029AE09EF16F0FF0E2B6E2BC0AF
:102C10002AF02A500101206F201F000120C16EF10F
:102C200073EC08F02B500101206F201F000120C120
:102C30006EF173EC08F0BEEF16F06EC021F16DC0BE
:102C400020F121EC08F0FF0E0101726FF20E716F9E
:102C5000000185EC07F0716A0101236BA60E226F5B
:102C6000256B060E246F0001FCEC14F00101236BB0
:102C7000320E226F256B060E246F0001FCEC14F05F
:102C8000ADC022F122C16EF173EC08F0ACC06EF160
:102C900073EC08F00E0E01012027000E2123000125
:102CA000B3EC07F001012153D8B403D0000168EF61
:102CB00016F00001010120513B08D8B003D00001FB
:102CC00068EF16F000010101216B3C0E206F00013E
:102CD000050E0101746F000120C175F179EC07F058
:102CE00021C122F1060E0101746F000122C175F1AC
:102CF00079EC07F00101746B240E756F000179EC1B
:102D000007F0000C21EC08F02AC0C3F02BC0C4F07F
:102D100001011F6B1E6B7052D8B403D0000197EFF6
:102D200016F000016F501C08D8B09FEF16F01C0E73
:102D30006F5C01011E6F000E70581F6F0001080EBE
:102D400001011E250001E86F000E01011F21000195
:102D5000E96F140EE825C16F000EE921C26F010171
:102D6000216B206B00018AEC14F0080EAD6FAC6B88
:102D7000110EAE6F60EC15F0CCEF15F01DEC16F0F7
:102D8000000C299629942988080EAD6FAC6B110EA2
:102D9000AE6FB86B440EB76FBA6B430EB96F0101DB
:102DA000216B1C0E206F00018AEC14F0010E010152
:102DB0006E6F000173EC08F0010E01016E6F0001EF
:102DC00073EC08F0060E01016E6F000173EC08F061
:102DD00001016E6B000173EC08F00101216BFF0E25
:102DE000206F0001B3EC14F0040E01011E6F00010E
:102DF000EAEC14F00101216B190E206F0001B3EC15
:102E000014F00C0E01011E6F0001EAEC14F0010138
:102E1000236B320E226F256B060E246F0001FCEC33
:102E200014F070500108D8A025EF17F0D8A41EEFB9
:102E300017F06F500708D8A025EF17F001016E6B4F
:102E4000000173EC08F011EF17F0630E01016E6FD3
:102E5000000173EC08F0820E01016E6F000173EC4B
:102E600008F0530E01016E6F000173EC08F0630E61
:102E700001016E6F000173EC08F0350E01016E6FF9
:102E8000000173EC08F0010E01016E6F000173EC9C
:102E900008F001011A510F0B1E6F00011EC16EF1E7
:102EA00073EC08F03D0E01016E6F000173EC08F049
:102EB000070E01016E6F000173EC08F0010E0101B5
:102EC0006E6F000173EC08F00101236B320E226F6C
:102ED000256B060E246F0001FCEC14F00C0E0101B2
:102EE0006E6F000173EC08F02998036A360EE96EE4
:102EF00003C0EAFFECCF1FF1ED52EFCF1EF11FC16F
:102F000021F11EC120F1C8EC13F002C01DF101C077
:102F10001CF11DC164F11CC163F150EC12F001C041
:102F20001BF12988060E01011B251E6F00011EC121
:102F30006EF173EC08F0000E81BA010E000AD8A4FD
:102F4000B8EF17F001011E6B000101011E510001D5
:102F500004EC01F00009D8B4B6EF17F001011E2B04
:102F60006E6F000173EC08F0A5EF17F0CCEF17F0CF
:102F700001011E6B000101011E51000110EC01F066
:102F80000009D8B4CCEF17F001011E2B6E6F0001C1
:102F900073EC08F0BBEF17F01DC164F11CC163F1C5
:102FA00050EC12F001011A510308D8B403D000010B
:102FB00002EF18F00001360E01016E6F000173EC94
:102FC00008F0040E01016E6F000173EC08F0010EB1
:102FD0000101216F090E206F0001B3EC14F0320ED5
:102FE00001016E6F000173EC08F0040E01016E6FB9
:102FF000000173EC08F00101216BFB0E206F000152
:10300000B3EC14F0370E01016E6F000173EC08F0A1
:10301000040E01016E6F000173EC08F0010E010156
:103020006E6F000173EC08F00F0E01016E6F00016E
:1030300073EC08F0030E01016E6F000173EC08F0F1
:10304000060E01016E6F000173EC08F0FF0E010126
:103050006E6F000173EC08F001011A511308D8B427
:1030600003D000014DEF18F00001EA6AA60EE96EE8
:10307000010EE26E030EE16E060E016EE6CFEEFF6C
:10308000012E3EEF18F00CC1B6F00BC1B5F00AC12D
:10309000B4F009C1B3F061EF18F0060E016EEA6AF0
:1030A000A60EE96EFF0EEE6E012E52EF18F0040E22
:1030B000016EEA6AB30EE96EFF0EEE6E012E5CEF52
:1030C00018F082EC16F014EF19F0EC53D8A4BDEF11
:1030D00018F01C6A1B6A1A6A196A036A360EE96ECE
:1030E00003C0EAFFECCF1BF1ED52EFCF1AF11BC189
:1030F00021F11AC120F1C8EC13F002C019F101C08E
:1031000018F1F66BF56B0101216BED0E206F236B4F
:10311000226B000136EC07F00101216BEF0E206FEE
:10312000236B226B000136EC07F019C11BF118C1AB
:103130001AF167EF14F002C01BF101C01AF101018E
:103140001A511F0B006E1B51000B036E0050140F21
:103150000001F16F000E0320F26FF2C0F4F0F1C035
:10316000F3F019C100F118C1FFF0F4C002F1F3C08F
:1031700001F1010EEC6F25EF19F0EC2DC2EF18F004
:10318000CCEF18F0EC510308D8B4CCEF18F0EC51A8
:103190001308D8A425EF19F00101216BED0E206F63
:1031A0000001F2C023F1F1C022F136EC07F0015228
:1031B000D8B425EF19F001011A6B000101011A5171
:1031C0000001F2EC00F001011A2B00019EA8E6EFCD
:1031D00018F0AD6E120E01011A5DD8B403D00001D3
:1031E000DEEF18F0060E1B6F00012E0E9EA8F6EF04
:1031F00018F0AD6E01011B2F02D004D000010001B8
:10320000F5EF18F0010E16262B6A00012BC02AF0EC
:103210002A52D8A40FEF19F0299010EF19F0298045
:10322000ECC01AF1C1EF16F0F2510408D8A025EF56
:1032300019F0D8A421EF19F0F151AF08D8A025EF6B
:1032400019F0F351F127F451F223EC513008D8B4BE
:103250002FEF19F0EC511308D8A464EF19F0010115
:10326000216BEF0E206F236B140E226F000136ECE2
:1032700007F00152D8B460EF19F0F52BD8B4F62B53
:10328000F951F55DD8A452EF19F0FA51F65DD8A4C2
:1032900052EF19F0F4C0F2F0F3C0F1F0130EEC6F3E
:1032A00060EF19F0F851F65DD8A060EF19F0D8A4DE
:1032B0005FEF19F0F751F55DD8A060EF19F0EC6BF6
:1032C000010E016E66EF19F0000E016EDAEF3EF0AE
:1032D0000101206B216B0001010121511E5DD8B05D
:1032E00003D00001AAEF19F00001D8A481EF19F072
:1032F00001011D51205DD8A003D00001AAEF19F0F3
:103300000001010E0101686F1F0E676F000188EC5C
:103310000BF00152D8B4AAEF19F001011B511C1196
:10332000D8A403D00001A3EF19F0000101011C5142
:10333000036E1B511B2BD8B41C2BE96E000103C07C
:10334000EAFF1FC1EFFF0101202BD8B4212B0001A0
:103350006CEF19F001012051016E2151026E000144
:10336000000C01011C515E08D8A003D00001C1EF80
:1033700019F00001E70E01011C251C6F0001CEEFC2
:1033800019F001011C514508D8B003D00001CEEF5F
:1033900019F00001190E01011C27000101011C5147
:1033A000016E0001000C3D6A3C6A070E0101716F5D
:1033B0000001A6EC07F00150100B000AD8B4E8EFAA
:1033C00019F02E0E9EA8E2EF19F0AD6EE1EC10F0B0
:1033D0000101746B600E756F000179EC07F0070E48
:1033E0000101716F0001A6EC07F00101196B0001EA
:1033F00001C018F10101746B200E756F000179ECAA
:1034000007F038500101185DD8B403D0000112EF65
:103410001AF0000101011953D8A403D00001C2EF32
:103420001AF0000138C039F001011C6B000138C0EE
:103430001BF11BC13BF03A6A6EEC09F0120E010160
:10344000706F0001B6EC0AF001011C6B9C0E1B6F43
:103450001E6B120E1D6F000168EC19F0120E3A2659
:10346000000E3B226EEC09F09FC03DF09EC03CF088
:103470009C51010B000AD8B464EF1AF03D52D8A455
:1034800047EF1AF03C503F08D8B064EF1AF03D50B7
:103490000508D8A064EF1AF0D8A454EF1AF03C50F5
:1034A000EE08D8A064EF1AF0120E3C5E000E3D5AF2
:1034B000ADC021F1ACC020F1C8EC13F002C0ADF0FA
:1034C00001C0ACF07EEF1AF03D6A3C6A01011B6B53
:1034D000000101011B51000112EC00F001011B2B46
:1034E00000019EA871EF1AF0AD6E0D0E01011B5D7B
:1034F000D8B403D0000169EF1AF000019D514508CE
:10350000D8B08CEF1AF09D515E08D8A08CEF1AF05D
:103510009DC038F0AFEF1AF03D6A3C6A01011B6BA9
:10352000000101011B51000121EC00F001011B2BE6
:1035300000019EA899EF1AF0AD6E0D0E01011B5D02
:10354000D8B403D0000191EF1AF0010E38241B6F9C
:1035500000011BC11CF1B1EC19F001C038F0010EE3
:10356000385C01011B6F00011BC11CF1B1EC19F0AB
:1035700001C01AF1030E0101746F00011AC175F147
:1035800079EC07F03C52D8A4CDEF1AF03D52D8A404
:10359000CDEF1AF0000ECEEF1AF0010E016EF2EF31
:1035A0003EF0716A6E6A71C06DF06EC070F06DC0F1
:1035B0006FF02B6A2BC02AF02A52D8A4E3EF1AF03E
:1035C0002990E4EF1AF029800101726B716B000100
:1035D00085EC07F0000C010E0101686F560E676F55
:1035E000000188EC0BF00152D8B404EF1BF001018C
:1035F0005651555DD8B403D0000104EF1BF0000113
:10360000010E016E06EF1BF0000E016E000C010EA4
:103610000101686F200E676F000188EC0BF001520A
:10362000D8B441EF1BF0010E0101686F210E676FE6
:10363000000188EC0BF00152D8B441EF1BF00101FE
:10364000256B000120C124F124C127F10101266B63
:10365000036A21512611226F03502711236F0001A5
:103660001FC103F001011E51E96E000103C0EAFF12
:1036700023C1ECFFED5222C1EFFF010E016E43EFBB
:103680001BF0000E016E000C040E01011F6F030EF3
:103690001D25216F000E1E21226F000122C168F13D
:1036A00021C167F188EC0BF00152D8B490EF1BF008
:1036B000020E01011D25226F000E1E21236F000145
:1036C00023C168F122C167F188EC0BF00152D8B434
:1036D00090EF1BF0010E01011D25236F000E1E212E
:1036E000246F000124C168F123C167F188EC0BF05D
:1036F0000152D8B490EF1BF001011D51246F1E51EF
:10370000256F000125C168F124C167F188EC0BF039
:103710000152D8B490EF1BF0010E016E92EF1BF036
:10372000000E016E000C01011E511F11D8A403D020
:103730000001B0EF1BF00001010E0101686F200EC7
:10374000676F000188EC0BF00152D8B4B0EF1BF0AA
:1037500001011E51D8B41F071E07000193EF1BF093
:1037600001011E53D8B403D00001C4EF1BF00001C7
:1037700001011F53D8B403D00001C4EF1BF00001B6
:10378000010E016EC6EF1BF0000E016E000C030E61
:1037900001011A25E96E000E1B21EA6E0001EFCF30
:1037A0001CF11CC155F1EBEC1AF00152D8B411EF29
:1037B0001CF0020E01011A25E96E000E1B21EA6EB3
:1037C0000001EFCF1DF11DC155F1EBEC1AF00152D4
:1037D000D8B411EF1CF0010E01011A25E96E000E9C
:1037E0001B21EA6E0001EFCF1EF11EC155F1EBEC7B
:1037F0001AF00152D8B411EF1CF001011A51E96E10
:103800001B51EA6E0001EFCF1FF11FC155F1EBEC28
:103810001AF00152D8B411EF1CF0010E016E13EF33
:103820001CF0000E016EEEEF1CF001011D6B00019B
:10383000D1EC1AF001011A2D02D004D000010001D0
:103840002DEF1CF00001060E016EEA6AA60EE96E6D
:10385000FF0EEE6E012E28EF1CF00101216B010E10
:10386000206F00011EEC15F0080E0101216F206B86
:1038700000011EEC15F0060E01016E6F000173ECE5
:1038800008F0040E01016E6F000173EC08F00101F5
:103890001C6B00011AC11BF11CC121F11BC120F1DD
:1038A0001EEC15F00101236B320E226F256B060E04
:1038B000246F0001FCEC14F00101216B190E206F44
:1038C0000001B3EC14F00101236BA60E226F256BEF
:1038D000060E246F0001FCEC14F00101216BB30E05
:1038E000206F0001B3EC14F0080EAD6F060EAC6F44
:1038F0001DEC16F009EF1DF00101556B0001EBEC1A
:103900001AF00152D8B442EF1DF0010E0101556FBB
:103910000001EBEC1AF00152D8B442EF1DF0080E92
:103920000101556F0001EBEC1AF00152D8B442EFDF
:103930001DF00101556B0001EBEC1AF00152D8B4F7
:1039400042EF1DF0060E0101556F0001EBEC1AF07D
:103950000152D8B442EF1DF0040E0101556F000171
:10396000EBEC1AF00152D8B442EF1DF0010E010148
:103970001F6F180E1E6F000107EC1BF00152D8B428
:1039800042EF1DF001011C6BBB0E1B6F1E6B060E80
:103990001D6F000168EC19F001500210D8B442EF1D
:1039A0001DF001011E6BB30E1D6F000144EC1BF0F6
:1039B0000152D8B442EF1DF001011F6B060E1E6FBD
:1039C000000193EC1BF00152D8B442EF1DF001014D
:1039D0001B6B190E1A6F0001C7EF1BF00152D8B410
:1039E00042EF1DF00101182D02D004D000010001AA
:1039F0000FEF1DF0000101011953D8B403D00001ED
:103A00000FEF1DF00001020E01011A6F000115EF0A
:103A10001CF0010E016E44EF1DF042EF1DF001019C
:103A200018510208D8B403D0000142EF1DF0000184
:103A300001011953D8B403D0000142EF1DF0000179
:103A40002550B35DD8A441EF1DF02650B45DD8A435
:103A500041EF1DF02750B55DD8A441EF1DF028506F
:103A6000B65DD8A441EF1DF0EA6A2C0EE96EE26A59
:103A7000BB0EE16E060E016EE6CFEEFF012E3CEFAF
:103A80001DF0148C000E016E07EF3FF0010E0101D6
:103A9000686F1D0E676F000188EC0BF00152D8B4FF
:103AA00056EF1DF0010E016E58EF1DF0000E016E75
:103AB000000C01011A513E241C6F1B513F201D6F49
:103AC0003D5CD8B003D0000177EF1DF00001D8A411
:103AD00073EF1DF03C5001011C5DD8A003D0000124
:103AE00077EF1DF000011DC13DF01CC13CF04150BD
:103AF00001011A251C6F000E1B211D6F1D53D8B428
:103B000003D0000190EF1DF00001405001011C5D49
:103B1000D8A003D0000190EF1DF000011CC140F0BF
:103B200039EF1EF02990299A2B6A2BC02AF0450EF6
:103B30000101556F0001EBEC1AF00152D8B43DEFD2
:103B40001EF046EC1DF00152D8B43DEF1EF001010D
:103B50001F6BC10E1E6F000107EC1BF00152D8B4A1
:103B60003DEF1EF001011F6B020E1E6F000193EC72
:103B70001BF00152D8B43DEF1EF001011F6B020E85
:103B80001E6F000193EC1BF00152D8B43DEF1EF004
:103B900046EC1DF00152D8B43DEF1EF00101686BF8
:103BA000AE0E676F000188EC0BF00152D8B43DEF08
:103BB0001EF001011F6B020E1E6F000193EC1BF043
:103BC0000152D8B43DEF1EF001011E6BB30E1D6F04
:103BD000000144EC1BF00152D8B43DEF1EF001018E
:103BE0001E6BAF0E1D6F000144EC1BF00152D8B4E8
:103BF0003DEF1EF01950AF5DD8A40EEF1EF01A5025
:103C0000B05DD8A40EEF1EF01B50B15DD8A40EEF2E
:103C10001EF01C50B25DD8B41AEF1EF0AF3D3DEF60
:103C20001EF0B03D3DEF1EF0B13D3DEF1EF0B23D48
:103C30003DEF1EF02A3C3DEF1EF02B3C3DEF1EF009
:103C4000C253D8A429EF1EF0C1511408D8B03DEFDB
:103C50001EF0140EC15D0101186F000E0001C25963
:103C60000101196F000119C11BF118C11AF159EFB7
:103C70001DF0010E016E3FEF1EF0000E016E12EFFF
:103C80003FF03D5001011F5DD8B003D000015AEF55
:103C90001EF00001D8A456EF1EF001011E513C5C3D
:103CA000D8A003D000015AEF1EF00001000E016EF3
:103CB00069EF1EF01FC171F11EC170F13AEC09F0FD
:103CC0001FC13FF01EC13EF0416A41C040F0010EED
:103CD000016E000C0101216B226B236B000121ECB2
:103CE00008F001016A6B2A0E6B6F0001FAEC0AF012
:103CF0000152D8A480EF1EF04052D8B4D6EF1EF087
:103D000040C020F1010120512225246F000E232103
:103D1000256F1F51255DD8B003D00001A9EF1EF01B
:103D20000001D8A49DEF1EF001011E51245DD8B002
:103D300003D00001A9EF1EF00001010E0101216F67
:103D400022511E5D006E23511F59036E0050206FDB
:103D50000001416A01012051415CD8A003D000015B
:103D6000C2EF1EF00001420E4124E96EEA6AD8B0AB
:103D7000EA2AEFCF24F124C16EF173EC08F0412A56
:103D8000AAEF1EF0010120513E26000E3F222051D5
:103D90002227000E23232153D8A403D00001D4EFFF
:103DA0001EF00001D6EF1EF071EF1EF06E50705C39
:103DB000D8A0E8EF1EF0D8A4E3EF1EF06F506D5CC2
:103DC000D8B0E8EF1EF070C003F06F50EBEF1EF0BC
:103DD0006EC003F06D506D6E03C06EF00101225194
:103DE000016E2351026E0001000C29902B6A2BC03A
:103DF0002AF0140EC15D01011E6F000E0001C259B0
:103E000001011F6F040E1E5D1C6F000E1F591D6FF8
:103E100019500001AF5DD8A47CEF1FF01A50B05DBF
:103E2000D8A47CEF1FF01B50B15DD8A47CEF1FF02D
:103E30001C50B25DD8A47CEF1FF0080E0101556F35
:103E40000001EBEC1AF00152D8B47CEF1FF0010135
:103E5000556B0001EBEC1AF00152D8B47CEF1FF067
:103E6000010E01011F6F180E1E6F000107EC1BF001
:103E70000152D8B47CEF1FF03FC01BF13EC01AF1D5
:103E80001DC11FF11CC11EF193EC1BF01BC11FF1E2
:103E90001AC11EF141EC1EF02A3C7CEF1FF02B3CB6
:103EA0007CEF1FF060EC15F00101216B206B00012D
:103EB0001EEC15F0080E0101192719510708D8B09A
:103EC00003D000016AEF1FF000010101182BD8B4E4
:103ED000192B000119C121F118C120F11EEC15F0B8
:103EE0001DC11FF11CC11EF16AEC1EF01DEC16F085
:103EF000010E016E7EEF1FF0000E016E1BEF3FF012
:103F00003E503C5C006E3F503D58036E0050016EC9
:103F10000350026E0CEF22F001011F53D8A403D00E
:103F20000001B9EF1FF00001010E0101686F200EC2
:103F3000676F000188EC0BF00152D8B4B9EF1FF0A5
:103F40001EC103F001011D51E96E000103C0EAFF2B
:103F500001012051EF5CD8B403D00001B9EF1FF08C
:103F6000000101011D2BD8B41E2B1F0700018CEF8F
:103F70001FF001011F53D8B403D00001C5EF1FF09B
:103F80000001010E016EC7EF1FF0000E016E10EF71
:103F900020F001011C6B298A020E556F0001EBEC29
:103FA0001AF00152D8B499EF21F046EC1DF00152FD
:103FB000D8B499EF21F0060E0101556F0001EBEC2A
:103FC0001AF00152D8B499EF21F001011F6B0D0EC8
:103FD0001E6F000193EC1BF00152D8B499EF21F051
:103FE000010E01011E6F110E1D6F000144EC1BF04C
:103FF0000152D8B499EF21F001011F6B080E1E6F1A
:10400000000193EC1BF00152D8B499EF21F00101AB
:104010001E6B320E1D6F060E1F6F00018CEF1FF01E
:104020000152D8B499EF21F001011F6BCA0E1E6F27
:10403000000193EC1BF00152D8B499EF21F02998BC
:1040400029942986630E0101556F0001EBEC1AF0EB
:104050000152D8B499EF21F0820E0101556F000191
:10406000EBEC1AF00152D8B499EF21F0530E010194
:10407000556F0001EBEC1AF00152D8B499EF21F022
:10408000630E0101556F0001EBEC1AF00152D8B438
:1040900099EF21F0010E0101686F1A0E676F0001A0
:1040A00088EC0BF00152D8B4F6EF20F001011A3D74
:1040B00002D004D00001000161EF20F00001F6EF12
:1040C00020F0010E0101686F1B0E676F000188EC84
:1040D0000BF00152D8B4F6EF20F001011A51350867
:1040E000D8B403D0000189EF20F0000101011B2D9D
:1040F00002D004D00001000189EF20F00001010E80
:104100000101686F1C0E676F000188EC0BF0F4EF83
:1041100020F001011A513308D8B403D00001A5EFF3
:1041200020F0000101011B510408D8B403D00001A4
:10413000A5EF20F00001010E01011E6F0D0E1D6F95
:10414000000144EC1BF0F4EF20F001011A2D02D025
:1041500004D000010001C9EF20F0000101011B5152
:104160000408D8B403D00001C9EF20F00001010118
:104170001C510508D8B403D00001C9EF20F000019C
:1041800001011E6B210E1D6F000144EC1BF0F4EFCA
:1041900020F001011A510308D8B403D00001EDEF5B
:1041A00020F0000101011B510308D8A003D0000139
:1041B000EDEF20F0000101011C510508D8B403D037
:1041C0000001EDEF20F0000101011E6B250E1D6FB7
:1041D000000144EC1BF0F4EF20F001011F6B000123
:1041E0001BC11EF193EC1BF04AEF20F0EC2D28EFE1
:1041F00021F001011C510208D8B403D0000128EFBE
:1042000021F00001010EEA6E030EE96EE26AA60ECD
:10421000E16E060E016EE6CFEEFF012E0BEF21F0F0
:10422000B6C00CF1B5C00BF1B4C00AF1B3C009F1CE
:1042300014C1FEF013C1FDF012C1FCF011C1FBF07E
:10424000F4C0F2F0F3C0F1F0030EEC6F99EF21F03F
:10425000EC510308D8B432EF21F0EC511308D8A484
:1042600099EF21F001011C510508D8B403D00001D9
:1042700099EF21F00001A80EF86FC00EF76F010151
:104280001053D8B403D0000168EF21F00001010100
:104290000F53D8B403D0000168EF21F000010101F1
:1042A0000E51A808D8B003D0000168EF21F000013A
:1042B000D8A464EF21F001010D51BF08D8B003D09C
:1042C000000168EF21F000010EC1F8F00DC1F7F018
:1042D000F853D8A474EF21F0F7513B08D8A074EF3D
:1042E00021F0F86B3C0EF76FD890F831FA6FF73188
:1042F000F96FF66BF56BFEC01CF0FDC01BF0FCC047
:104300001AF0FBC019F0A4EC12F0ECEC12F034EC53
:1043100013F07CEC13F0166A0D0E9EA88DEF21F0C1
:10432000AD6E0A0E9EA892EF21F0AD6E300EEC6FCE
:10433000148E90EF22F02B6A2BC02AF0299E299030
:1043400001011F6BB90E1E6F000107EC1BF001523B
:10435000D8B494EF22F001011F6BB70E1E6F00015D
:1043600007EC1BF00152D8B494EF22F001011F6B4F
:10437000E80E1E6F000107EC1BF00152D8B494EF59
:1043800022F001011F6BEA0E1E6F000107EC1BF00B
:104390000152D8B494EF22F0E953D8A4D5EF21F01C
:1043A000E8510708D8B094EF22F0E9510508D8A0E9
:1043B00094EF22F0D8A4E2EF21F0E851C008D8A091
:1043C00094EF22F0EA51EB11D8B41CEF22F0E9C0CF
:1043D00022F1E8C021F1BEEC15F00101216BAF0E16
:1043E000206F000129EC15F00101216BB30E206F45
:1043F000000129EC15F001016F6B00014CEC08F095
:10440000110E01016F6F00014CEC08F03FC019F173
:104410003EC018F180EF1FF002C01BF101C01AF17D
:104420001BC11FF11AC11EF193EC1BF019C11FF142
:1044300018C11EF141EC1EF0EA53D8A424EF22F07B
:10444000EB53D8B42AEF22F02A3C94EF22F02B3C15
:1044500094EF22F001011D6B0001D1EC1AF02B6AE0
:104460002BC02AF02990B7510708D8A457EF22F0A3
:10447000B853D8A457EF22F00101216B1C0E206F16
:1044800000018AEC14F0080EE85D01011A6F000EBD
:104490000001E95901011B6F00011BC11FF11AC185
:1044A0001EF16AEC1EF082EC16F090EF22F0B7518C
:1044B0000D08D8A485EF22F0B853D8A485EF22F0D8
:1044C0002996299429880101216B1C0E206F000177
:1044D0008AEC14F001011A6B000101011A5100016C
:1044E00030EC00F001011A2B6D6F00019FEC08F019
:1044F0000C0E01011A5DD8B403D000016DEF22F05B
:10450000000182EC16F090EF22F0B7514408D8A4D5
:1045100090EF22F0B853D8A490EF22F0C9EF1FF02B
:10452000010E016E96EF22F0000E016E24EF3FF0B7
:1045300001011F51E96E2051EA6E2151EF24016EF5
:104540002251EC20036EE9060150EF6E000103C01A
:10455000ECFFE90601011F51E96E2051EA6E0001EE
:10456000ECCF24F1ED52EFCF23F101012451225D74
:10457000D8B003D00001DAEF22F00001D8A4CAEFCE
:1045800022F001012151235DD8A003D00001DAEF10
:1045900022F00001020E01011F25E96E000E20210C
:1045A000EA6E010EEE26D8B003D00001DAEF22F059
:1045B000EF2A0001000C948804009486040082987D
:1045C000949804008B969496A00E0101646F0001EC
:1045D00017EC0EF0D7C055F10101566B000155C123
:1045E00064F117EC0EF0D6C064F117EC0EF094985D
:1045F0000000948682A6FAEF22F00400000000007A
:104600000000948804009488040094860400829832
:10461000949804008B969496A10E0101646F00019A
:1046200017EC0EF0B4EF28F00101566B576B586B86
:10463000596B5A6B5B6B5C6B5D6B5E6B5F6B606B3E
:10464000616B626B636B646B656B666B566B0001D1
:10465000010156510408D8B003D0000154EF23F0F3
:104660000001010E0101686F550E676F000188ECB3
:104670000BF00152D8B454EF23F00101555120083A
:10468000D8A003D0000154EF23F0000101015551DF
:104690003D08D8A403D0000154EF23F0000101012C
:1046A000562B000128EF23F00101566B0001010198
:1046B00056510708D8B003D00001A6EF23F000013F
:1046C000010E0101686F550E676F000188EC0BF059
:1046D0000152D8B4A6EF23F0010155512008D8A00B
:1046E00003D00001A6EF23F0000101015551260877
:1046F000D8A403D00001A6EF23F00001570E01015A
:104700005625E96E010EEA6ED8B0EA2A55516008C6
:10471000D8A003D000019DEF23F000010101555105
:104720007A08D8B003D000019DEF23F00001010109
:104730005551DF0B0001A0EF23F00101555100019D
:10474000EF6E0101562B000157EF23F00101566B6C
:104750000001010156510408D8B003D00001D5EF83
:1047600023F00001010E0101686F550E676F000113
:1047700088EC0BF00152D8B4D5EF23F0010155516C
:104780002008D8A003D00001D5EF23F000010101DB
:1047900055513D08D8A403D00001D5EF23F0000106
:1047A0000101562B0001A9EF23F00101566B000116
:1047B000010156510708D8B003D0000127EF24F0BB
:1047C0000001010E0101686F550E676F000188EC52
:1047D0000BF00152D8B427EF24F001015551200805
:1047E000D8A003D0000127EF24F0000101015551AA
:1047F0002608D8A403D0000127EF24F000015F0EA3
:1048000001015625E96E010EEA6ED8B0EA2A55512B
:104810006008D8A003D000011EEF24F000010101C0
:1048200055517A08D8B003D000011EEF24F00001E2
:1048300001015551DF0B000121EF24F00101555119
:104840000001EF6E0101562B0001D8EF23F00101AA
:10485000566B0001010156510708D8B003D0000182
:1048600057EF24F00001570E01015625E96E010EA5
:10487000EA6ED8B0EA2A0001EFCF67F15F0E0101BE
:104880005625E96E010EEA6ED8B0EA2AEF50675D50
:10489000D8A403D0000152EF24F00001000E016EF5
:1048A000AAEF24F00101562B00012AEF24F00101A8
:1048B000566B0001010156510708D8B003D0000122
:1048C000A8EF24F000010A0E01015625676F0001D0
:1048D00067C1A9FFA86AA69CA69EA684F250006E96
:1048E000F29E0F01550EA76EAA0EA76EA6820001BA
:1048F000A6B278EF24F0A6940050F2120A0E01013D
:104900005625676F570E5625E96E010EEA6ED8B030
:10491000EA2A0001EFCF68F167C1A9FF68C1A8FFCB
:10492000A69CA69EA684F250006EF29E0F01550E24
:10493000A76EAA0EA76EA6820001A6B29DEF24F074
:10494000A6940050F2120101562B00015AEF24F0F8
:10495000010E016E4BEF2BF00101566B576B586B3C
:10496000596B5A6B5B6B5C6B5D6B5E6B566B0001DE
:10497000010156510408D8B003D00001E4EF24F03F
:104980000001010E0101686F550E676F000188EC90
:104990000BF00152D8B4E4EF24F001015551200886
:1049A000D8A003D00001E4EF24F00001010155512B
:1049B0003D08D8A403D00001E4EF24F00001010178
:1049C000562B0001B8EF24F00101566B00010101E4
:1049D00056510708D8B003D0000136EF25F000018A
:1049E000010E0101686F550E676F000188EC0BF036
:1049F0000152D8B436EF25F0010155512008D8A056
:104A000003D0000136EF25F00001010155513D08AA
:104A1000D8A403D0000136EF25F00001570E0101A4
:104A20005625E96E010EEA6ED8B0EA2A55516008A3
:104A3000D8A003D000012DEF25F000010101555150
:104A40007A08D8B003D000012DEF25F00001010154
:104A50005551DF0B000130EF25F0010155510001E8
:104A6000EF6E0101562B0001E7EF24F001015751D1
:104A70003008D8B403D0000182EF25F00001010115
:104A800058513508D8B403D0000182EF25F0000159
:104A9000010159513408D8B403D0000182EF25F048
:104AA000000101015A513008D8B403D0000182EF4F
:104AB00025F0000101015B513808D8B403D0000192
:104AC00082EF25F0000101015C513608D8B403D013
:104AD000000182EF25F0000101015D513508D8B4D5
:104AE00003D0000182EF25F0000101015E51320880
:104AF000D8B403D0000182EF25F00001010E016E51
:104B0000DAEF25F00101566B00010101565107084B
:104B1000D8B003D00001D8EF25F00001570E0101F5
:104B20005625E96E010EEA6ED8B0EA2AEF50200849
:104B3000D8B403D00001B1EF25F000010A0E010145
:104B40005625606F000160C1A9FFA69CA69EA680A5
:104B5000A850000AD8A4B1EF25F0010E016EDAEFDB
:104B600025F0570E01015625E96E010EEA6ED8B008
:104B7000EA2A0001EFCF5FF10A0E01015625606FAE
:104B8000000160C1A9FFA69CA69EA680A8500101B5
:104B90005F5DD8A403D00001D3EF25F00001000E23
:104BA000016EDAEF25F00101562B000185EF25F0AB
:104BB000010E016E8DEF2BF001015E5160030001CB
:104BC000F3CF01F0F4CF00F001016103F3500026B0
:104BD0005F516003F3500020026E000186EF26F063
:104BE0000101586B596B5A6B5B6B5C6B5D6B5B6B5C
:104BF0005A6B000101015B53D8B403D0000130EFC0
:104C000026F0000101015A510408D8B003D0000178
:104C100030EF26F00001010E0101686F570E676F3B
:104C2000000188EC0BF00152D8B430EF26F00101FE
:104C300057512008D8A003D0000130EF26F0000122
:104C4000010157513D08D8A403D0000130EF26F0F0
:104C5000000101015A2BD8B45B2B0001FAEF25F0BB
:104C600001015B6B5A6B000101015B53D8B403D0A7
:104C7000000199EF26F0000101015A510408D8B053
:104C800003D0000199EF26F00001010E0101686FC9
:104C9000570E676F000188EC0BF00152D8B499EF02
:104CA00026F0010157512008D8A003D0000199EF48
:104CB00026F00001010157512608D8A403D00001B5
:104CC00099EF26F00001010157512F08D8A003D019
:104CD000000192EF26F00001010157513908D8B0C8
:104CE00003D0000192EF26F00001300E0101575D64
:104CF0005C6F5D6B000159C15FF158C15EF101014C
:104D0000616B0A0E606F0001DCEF25F002C05FF1FD
:104D100001C05EF101015C515E25586F5D515F215C
:104D2000596F000101015A2BD8B45B2B000134EFFD
:104D300026F001015851016E5951026E0001000C1C
:104D40000F0E0101581758510908D8B003D00001BF
:104D5000B6EF26F00001300E01015825596F000111
:104D600059C16DF19FEC08F0BFEF26F0370E01013D
:104D70005825596F000159C16DF19FEC08F0000CE6
:104D800001015639576F0F0E5717000157C158F1DF
:104D9000A0EC26F056C158F1A0EC26F0000C55C14D
:104DA000A9FFA69CA69EA680A8500008D8B0EEEF4A
:104DB00026F055C1A9FFA69CA69EA680A85004086F
:104DC000D8A0EEEF26F055C1A9FFA69CA69EA6800E
:104DD000A850030F0101576F586B000155C1A9FF7F
:104DE000A69CA69EA680A8500408D8B00DEF27F078
:104DF00055C1A9FFA69CA69EA680A8500608D8A0CB
:104E00000DEF27F055C1A9FFA69CA69EA680A8502D
:104E1000FC0F0101576F586B000155C1A9FFA69CFB
:104E2000A69EA680A8500708D8A422EF27F055C157
:104E3000A9FFA69CA69EA680A850010F0101576F4E
:104E4000586B000155C1A9FFA69CA69EA680A8503C
:104E50000808D8A437EF27F055C1A9FFA69CA69E45
:104E6000A680A850FB0F0101576F586B000101018C
:104E70005751016E5851026E0001000C55C1A9FF37
:104E8000A69CA69EA680A8500108D8B452EF27F091
:104E900055C1A9FFA69CA69EA680A8500808D8A424
:104EA00058EF27F0290E016E000E026EA6EF27F0D4
:104EB00055C1A9FFA69CA69EA680A8500208D8B4FA
:104EC0006CEF27F055C1A9FFA69CA69EA680A8500E
:104ED0000308D8A472EF27F02A0E016E000E026EAE
:104EE000A6EF27F055C1A9FFA69CA69EA680A850B4
:104EF0000408D8B486EF27F055C1A9FFA69CA69E4A
:104F0000A680A8500708D8A48CEF27F02B0E016EBE
:104F1000000E026EA6EF27F055C1A9FFA69CA69E23
:104F2000A680A8500508D8B4A0EF27F055C1A9FF66
:104F3000A69CA69EA680A8500608D8A4A6EF27F097
:104F4000280E016E000E026EA6EF27F0000C006A1C
:104F500041EC0EF094980000948682A6ADEF27F005
:104F600004000000000000009488040054EF39F0B1
:104F7000010E0101356F010E366F010E376F386B70
:104F8000010E396F010E3A6F010E3B6F010E3C6F3F
:104F9000010E3D6F3E6B010E3F6F010E406F416B86
:104FA000010E426F010E436F446B010E456F010EFF
:104FB000466F476B010E486F010E496F4A6B010E39
:104FC0004B6F010E4C6F4D6B010E4E6F010E4F6F0C
:104FD000506B010E516F010E526F536B010E546FE7
:104FE0002B6A00012BC02AF02A52D8A4FBEF27F02D
:104FF0002990FCEF27F02980298A470E0101556F7F
:105000000001EBEC1AF00152D8B458EF39F0450E1C
:105010000101556F0001EBEC1AF00152D8B458EFC2
:1050200039F0540E0101556F0001EBEC1AF00152FA
:10503000D8B458EF39F0200E0101556F0001EBECA8
:105040001AF02F0E0101556F0001EBEC1AF001016F
:105050001D6B000101011D510B08D8B003D00001E8
:1050600066EF28F00001010E0101686F210E676FE5
:10507000000188EC0BF00152D8B466EF28F0010172
:1050800021512008D8A003D0000166EF28F00001CC
:10509000010121513F08D8A403D0000166EF28F098
:1050A0000001070E01011D25016E036AD8B0032A15
:1050B0000150D40FE96E000E0320EA6E000121C1F9
:1050C000EFFF01011D2B00012AEF28F001011D5106
:1050D0000B08D8B003D0000183EF28F00001070EC1
:1050E00001011D25016E036AD8B0032A0150D40FB7
:1050F000E96E000E0320EA6EEF6A000101011D2B2C
:10510000000166EF28F070EC0EF00152D8B48BEF7E
:1051100028F08EEF28F0DB6B70EC0EF02B6A2BC0C2
:105120002AF02990706A280E6F6EE753D8A4B2EF68
:1051300028F00101556B00010101555100014FECB0
:1051400000F00101552B6D6F00019FEC08F01F0E60
:105150000101555DD8B403D000019CEF28F0000197
:1051600054EF39F0DBEF22F0D451D511D8B452EF1F
:1051700039F0010E006E41EC0EF001C01FF1D45168
:10518000D8B4D507D407DA51010B000AD8B44CEFD4
:1051900039F001011F514008D8B403D000014CEF91
:1051A00039F00001D451D511D8B44CEF39F0010ECB
:1051B000006E41EC0EF001C01FF1D451D8B4D507F8
:1051C000D407300E01011F5D206F1F514008D8A089
:1051D00003D00001F2EF28F00001370E01011F5D3E
:1051E000206F00010101202D02D004D00001000138
:1051F000E1EF2AF00001010E0101556F000104ECFE
:105200000DF003C02CF102C02BF101C02AF100C047
:1052100029F101011D6B000101011D511F08D8B0CA
:1052200003D000015AEF29F000012CC130F12BC14D
:105230002FF12AC12EF129C12DF1350E01011D25B5
:10524000E96E010EEA6ED8B0EA2A000130C15BF1C6
:105250002FC15AF12EC159F12DC158F101011D5133
:10526000576FD8A403D0000145EF29F00001D89072
:1052700001015B335A3359335833572F02D004D0CE
:105280000001000137EF29F0000101015851010B25
:10529000006E5951000B016E5A51000B026E5B51AA
:1052A000000B036E000100C0EFFF01011D2B000188
:1052B0000CEF29F0030E01011D6F000101011D51CA
:1052C0000608D8B003D00001DFEF29F0000101018A
:1052D0001D51040DF350350FE96E010EEA6ED8B082
:1052E000EA2AEF52D8A403D000017BEF29F0000195
:1052F000310E7CEF29F0300E0101576F000157C1CC
:105300006EF173EC08F001011D51040DF350010F13
:10531000350FE96E010EEA6ED8B0EA2AEF52D8A432
:1053200003D0000198EF29F00001310E99EF29F028
:10533000300E0101576F000157C16EF173EC08F098
:1053400001011D51040DF350020F350FE96E010EDE
:10535000EA6ED8B0EA2AEF52D8A403D00001B5EF24
:1053600029F00001310EB6EF29F0300E0101576F20
:10537000000157C16EF173EC08F001011D51040DDD
:10538000F350030F350FE96E010EEA6ED8B0EA2A2A
:10539000EF52D8A403D00001D2EF29F00001310E62
:1053A000D3EF29F0300E0101576F000157C16EF1A4
:1053B00073EC08F001011D2B00015EEF29F0000ED7
:1053C00081BA010E000AD8A46AEF2AF001011D6B10
:1053D000000101011D510108D8B003D000016AEF9E
:1053E0002AF0000101011D51040DF350350FE96E43
:1053F000010EEA6ED8B0EA2AEF52D8A403D0000119
:1054000006EF2AF00001310E07EF2AF0300E0101FD
:10541000576F000157C16EF173EC08F001011D5187
:10542000040DF350010F350FE96E010EEA6ED8B08E
:10543000EA2AEF52D8A403D0000123EF2AF000019A
:10544000310E24EF2AF0300E0101576F000157C1D1
:105450006EF173EC08F001011D51040DF350020FC1
:10546000350FE96E010EEA6ED8B0EA2AEF52D8A4E1
:1054700003D0000140EF2AF00001310E41EF2AF085
:10548000300E0101576F000157C16EF173EC08F047
:1054900001011D51040DF350030F350FE96E010E8C
:1054A000EA6ED8B0EA2AEF52D8A403D000015DEF2B
:1054B0002AF00001310E5EEF2AF0300E0101576F25
:1054C000000157C16EF173EC08F001011D2B0001C2
:1054D000E9EF29F0070E01011D6F1D51040DF35076
:1054E000350FE96E010EEA6ED8B0EA2AEF52D8A461
:1054F00003D0000180EF2AF00001310E81EF2AF085
:10550000300E0101576F000157C16EF173EC08F0C6
:1055100001011D51040DF350010F350FE96E010E0D
:10552000EA6ED8B0EA2AEF52D8A403D000019DEF6A
:105530002AF00001310E9EEF2AF0300E0101576F64
:10554000000157C16EF173EC08F001011D51040D0B
:10555000F350020F350FE96E010EEA6ED8B0EA2A59
:10556000EF52D8A403D00001BAEF2AF00001310EA7
:10557000BBEF2AF0300E0101576F000157C16EF1E9
:1055800073EC08F001011D51040DF350030F350FAA
:10559000E96E010EEA6ED8B0EA2AEF52D8A403D021
:1055A0000001D7EF2AF00001310ED8EF2AF0300EBB
:1055B0000101576F000157C16EF173EC08F04AEF1B
:1055C00039F0010120510208D8B403D000010AEFDC
:1055D0002BF00001080EA96EA69CA69EA680A850DE
:1055E000000AD8A408EF2BF00101556B000101015E
:1055F0005551000167EC00F00009D8B408EF2BF01A
:105600000101552B6E6F000173EC08F0F7EF2AF0E3
:105610004AEF39F0010120510308D8B403D000014A
:1056200033EF2BF00001080EA96EA69CA69EA68063
:10563000A8500108D8A431EF2BF00101556B0001EF
:1056400001015551000167EC00F00009D8B431EFB9
:105650002BF00101552B6E6F000173EC08F020EF69
:105660002BF04AEF39F0010120510408D8B403D0DF
:10567000000140EF2BF00001010E156E4AEF39F0EA
:10568000010120510608D8B403D0000182EF2BF0AD
:10569000000114EF23F001C01DF101011D2D02D006
:1056A00004D0000100016CEF2BF000010101556BEB
:1056B000000101015551000173EC00F00009D8B45C
:1056C0006AEF2BF00101552B6E6F000173EC08F0AF
:1056D00059EF2BF080EF2BF00101556B0001010118
:1056E0005551000182EC00F00009D8B480EF2BF096
:1056F0000101552B6E6F000173EC08F06FEF2BF07A
:105700004AEF39F0010120510708D8B403D0000155
:10571000A4EF2BF00001ACEF24F001C01DF101015A
:105720001D53D8A403D000019AEF2BF00001310ED5
:105730009BEF2BF0300E0101556F000155C16EF14A
:1057400073EC08F04AEF39F0010120510808D8B491
:1057500003D000010BEF2CF000010101646B00018C
:105760001CC063F150EC12F02E0E01016E6F0001AF
:1057700073EC08F00101646B00011BC063F150EC95
:1057800012F02E0E01016E6F000173EC08F00101A2
:10579000646B00011AC063F150EC12F02E0E01018F
:1057A0006E6F000173EC08F00101646B000119C019
:1057B00063F150EC12F01752D8A4F5EF2BF0010171
:1057C000556B00010101555100018FEC00F00009FB
:1057D000D8B4F3EF2BF00101552B6E6F000173EC81
:1057E00008F0E2EF2BF009EF2CF00101556B0001FE
:1057F0000101555100019BEC00F00009D8B409EFFC
:105800002CF00101552B6E6F000173EC08F0F8EFDE
:105810002BF04AEF39F0010120510908D8B403D028
:105820000001BAEF2DF00001A96A36C0A8FFA69CBE
:10583000A69EA684F250006EF29E0F01550EA76E32
:10584000AA0EA76EA6820001A6B224EF2CF0A694A1
:105850000050F212010EA96E37C0A8FFA69CA69EAA
:10586000A684F250006EF29E0F01550EA76EAA0E8E
:10587000A76EA6820001A6B23BEF2CF0A6940050C2
:10588000F212F0EC25F002C056F101C055F1020E03
:10589000A96E55C1A8FFA69CA69EA684F250006ED4
:1058A000F29E0F01550EA76EAA0EA76EA6820001EA
:1058B000A6B258EF2CF0A6940050F212F0EC25F0AE
:1058C00002C056F101C055F1030EA96E55C1A8FFE3
:1058D000A69CA69EA684F250006EF29E0F01550E65
:1058E000A76EAA0EA76EA6820001A6B275EF2CF0D5
:1058F000A6940050F212F0EC25F002C056F101C05F
:1059000055F1040EA96E55C1A8FFA69CA69EA684BB
:10591000F250006EF29E0F01550EA76EAA0EA76EF2
:10592000A6820001A6B292EF2CF0A6940050F212CB
:10593000F0EC25F002C056F101C055F1050EA96E3C
:1059400055C1A8FFA69CA69EA684F250006EF29EAA
:105950000F01550EA76EAA0EA76EA6820001A6B271
:10596000AFEF2CF0A6940050F212F0EC25F002C03C
:1059700056F101C055F1130EA96E55C1A8FFA69CA2
:10598000A69EA684F250006EF29E0F01550EA76EE1
:10599000AA0EA76EA6820001A6B2CCEF2CF0A694A8
:1059A0000050F212F0EC25F002C056F101C055F1A2
:1059B000140EA96E55C1A8FFA69CA69EA684F250FF
:1059C000006EF29E0F01550EA76EAA0EA76EA6825C
:1059D0000001A6B2E9EF2CF0A6940050F212F0EC10
:1059E00025F002C056F101C055F1150EA96E55C142
:1059F000A8FFA69CA69EA684F250006EF29E0F0100
:105A0000550EA76EAA0EA76EA6820001A6B206EFDB
:105A10002DF0A6940050F212F0EC25F002C056F1E1
:105A200001C055F1160EA96E55C1A8FFA69CA69EF1
:105A3000A684F250006EF29E0F01550EA76EAA0EBC
:105A4000A76EA6820001A6B223EF2DF0A694005007
:105A5000F212F0EC25F002C056F101C055F1170E1C
:105A6000A96E55C1A8FFA69CA69EA684F250006E02
:105A7000F29E0F01550EA76EAA0EA76EA682000118
:105A8000A6B240EF2DF0A6940050F212F0EC25F0F3
:105A900002C056F101C055F1180EA96E55C1A8FFFC
:105AA000A69CA69EA684F250006EF29E0F01550E93
:105AB000A76EAA0EA76EA6820001A6B25DEF2DF01A
:105AC000A6940050F212F0EC25F002C056F101C08D
:105AD00055F1190EA96E55C1A8FFA69CA69EA684D5
:105AE000F250006EF29E0F01550EA76EAA0EA76E21
:105AF000A6820001A6B27AEF2DF0A6940050F21211
:105B0000F0EC25F002C056F101C055F11A0EA96E55
:105B100055C1A8FFA69CA69EA684F250006EF29ED8
:105B20000F01550EA76EAA0EA76EA6820001A6B29F
:105B300097EF2DF0A6940050F21203EC02F001C092
:105B400055F1060EA96E55C1A8FFA69CA69EA68477
:105B5000F250006EF29E0F01550EA76EAA0EA76EB0
:105B6000A6820001A6B2B2EF2DF0A6940050F21268
:105B70004AEF39F0010120510A08D8B403D00001DE
:105B800046EF2FF00001010E926E81EC03F0040E3F
:105B900001011E6F000101011E510708D8B003D09A
:105BA000000182EF2EF000011EC157F1B4EC0DF0A0
:105BB00001012C6B2B6B000102C02AF101C029F1FD
:105BC00001011D6B000101011D511F08D8B003D058
:105BD000000131EF2EF000012CC130F12BC12FF16B
:105BE0002AC12EF129C12DF1350E01011D25E96EC5
:105BF000010EEA6ED8B0EA2A000130C15BF12FC174
:105C00005AF12EC159F12DC158F101011D51576FA3
:105C1000D8A403D000011CEF2EF00001D8900101A0
:105C20005B335A3359335833572F02D004D0000115
:105C300000010EEF2EF0000101015851010B006E22
:105C40005951000B016E5A51000B026E5B51000B53
:105C5000036E000100C0EFFF01011D2B0001E3EF07
:105C60002DF001013653D8A403D000013CEF2EF0F3
:105C70000001310E3DEF2EF0300E0101556F000195
:105C800055C16EF173EC08F001013753D8A403D06D
:105C900000014FEF2EF00001310E50EF2EF0300ECC
:105CA0000101556F000155C16EF173EC08F001015F
:105CB0003853D8A403D0000162EF2EF00001310E5A
:105CC00063EF2EF0300E0101556F000155C16EF1EA
:105CD00073EC08F001013D53D8A403D0000175EF27
:105CE0002EF00001310E76EF2EF0300E0101556FCF
:105CF000000155C16EF173EC08F001011E2B00018B
:105D0000CBEF2DF0000E81BA010E000AD8A444EFAB
:105D10002FF0010E01011E6F000101011E5102084A
:105D2000D8B003D0000144EF2FF000011EC157F19D
:105D3000B4EC0DF001012C6B2B6B000102C02AF1B9
:105D400001C029F101011D6B000101011D511F0856
:105D5000D8B003D00001F3EF2EF000012CC130F1D8
:105D60002BC12FF12AC12EF129C12DF1350E0101D0
:105D70001D25E96E010EEA6ED8B0EA2A000130C195
:105D80005BF12FC15AF12EC159F12DC158F101011A
:105D90001D51576FD8A403D00001DEEF2EF0000193
:105DA000D89001015B335A3359335833572F02D0FF
:105DB00004D000010001D0EF2EF000010101585184
:105DC000010B006E5951000B016E5A51000B026E0F
:105DD0005B51000B036E000100C0EFFF01011D2BA2
:105DE0000001A5EF2EF001013653D8A403D0000125
:105DF000FEEF2EF00001310EFFEF2EF0300E01010C
:105E0000556F000155C16EF173EC08F00101375375
:105E1000D8A403D0000111EF2FF00001310E12EFD2
:105E20002FF0300E0101556F000155C16EF173EC7A
:105E300008F001013853D8A403D0000124EF2FF05B
:105E40000001310E25EF2FF0300E0101556F0001DA
:105E500055C16EF173EC08F001013D53D8A403D095
:105E6000000137EF2FF00001310E38EF2FF0300E28
:105E70000101556F000155C16EF173EC08F001018D
:105E80001E2B00018DEF2EF04AEF39F00101205159
:105E90000C08D8B403D0000167EF2FF00001060E04
:105EA000A96EA86AA69CA69EA684F250006EF29ED9
:105EB0000F01550EA76EAA0EA76EA6820001A6B20C
:105EC0005FEF2FF0A6940050F2124AEF39F0010173
:105ED00020510D08D8B403D0000185EF30F0000147
:105EE000010E926E01011D6B000101011D5112088E
:105EF000D8B003D0000198EF2FF00001350E01015A
:105F00001D25016E010E036ED8B0032A0150556F96
:105F1000000103C056F1F0EC25F056C1EAFF55C16F
:105F2000E9FF01C0EFFF01011D2B000175EF2FF00C
:105F3000040E01011E6F000101011E510708D8B0B7
:105F400003D000010AEF30F000011EC157F1B4EC9C
:105F50000DF002C026F101C025F101012551F00B21
:105F6000556F2651566F1E51030DF350F60F350F26
:105F7000E96E010EEA6ED8B0EA2AEF50080DF35030
:105F800055255A6F000E56215B6F1E51030DF350BD
:105F9000F50F350FE96E010EEA6ED8B0EA2AEF5020
:105FA000040DF3505A255F6F000E5B21606F1E5188
:105FB000030DF350F40F350FE96E010EEA6ED8B001
:105FC000EA2AD890EF34006E5F25646F000E6021DE
:105FD000656F2551010B006E2651000B036E0050BA
:105FE0006425276F03506521286F000181EC03F0C1
:105FF00028C155F10101566B00011EC15CF155C16C
:106000005DF127C15EF1D7EC03F001011E2B000109
:106010009CEF2FF0000E81BA010E000AD8A483EF86
:1060200030F0010E01011E6F000101011E51020836
:10603000D8B003D0000183EF30F000011EC157F14A
:10604000B4EC0DF002C026F101C025F1010125518B
:10605000F00B556F2651566F1E51030DF3500B0F69
:10606000350FE96E010EEA6ED8B0EA2AEF50080D3E
:10607000F35055255A6F000E56215B6F1E51030DCC
:10608000F3500A0F350FE96E010EEA6ED8B0EA2A16
:10609000EF50040DF3505A255F6F000E5B21606FC7
:1060A0001E51030DF350090F350FE96E010EEA6E14
:1060B000D8B0EA2AD890EF34006E5F25646F000EE6
:1060C0006021656F2551010B006E2651000B036E98
:1060D00000506425276F03506521286F000181EC73
:1060E00003F028C155F10101566B00011EC15CF19E
:1060F00055C15DF127C15EF1D7EC03F001011E2B04
:10610000000115EF30F04AEF39F0010120510E087F
:10611000D8B403D000011AEF31F00001010E926EE5
:1061200081EC03F0F0EC25F002C056F101C055F10E
:10613000080EA96E55C1A8FFA69CA69EA684F25083
:10614000006EF29E0F01550EA76EAA0EA76EA682D4
:106150000001A6B2A9EF30F0A6940050F212080E8A
:10616000A96EA69CA69EA680A8500108D8A4C5EF3B
:1061700030F0110E01015C6FFF0E5D6F200E5E6F3F
:106180000001D7EC03F018EF31F0110E01015C6F44
:10619000FF0E5D6F5E6B0001D7EC03F0010E926E97
:1061A00081EC03F0010E01011E6F000101011E517F
:1061B0000708D8B003D0000118EF31F000011EC16C
:1061C00057F1B4EC0DF001012C6B2B6B000102C0F8
:1061D0002AF101C029F101012951E00B256F2A5153
:1061E000266F29510F0B276F2A51000B286F27515B
:1061F0002525296F285126212A6F2B6B2C6B000136
:1062000081EC03F02AC156F12BC157F12CC158F192
:106210000101596B00011EC15CF156C15DF129C13C
:106220005EF1D7EC03F001011E2B0001D6EF30F038
:106230004AEF39F0010120510F08D8B403D0000112
:106240003DEF31F000019AEC05F0120EA96EA86A3C
:10625000A69CA69EA684F250006EF29E0F01550EDB
:10626000A76EAA0EA76EA6820001A6B235EF31F086
:10627000A6940050F2124AEF39F0010120511008A3
:10628000D8B403D0000156EF31F00001090EA96E19
:10629000A69CA69EA680A8500101556F646B0001C4
:1062A00055C163F150EC12F04AEF39F00101205171
:1062B0001108D8B403D000017EEF31F00001F0ECFA
:1062C00025F002C056F101C055F1090EA96E55C165
:1062D000A8FFA69CA69EA684F250006EF29E0F0117
:1062E000550EA76EAA0EA76EA6820001A6B276EF83
:1062F00031F0A6940050F2124AEF39F0010120511A
:106300001208D8B403D00001A7EF31F00001120E3B
:10631000A96EA69CA69EA680A850000AD8A4A5EFA8
:1063200031F00101556B000101015551000167EC8D
:1063300000F00009D8B4A5EF31F00101552B6E6FC4
:10634000000173EC08F094EF31F04AEF39F00101ED
:1063500020511308D8B403D00001D0EF31F0000170
:10636000120EA96EA69CA69EA680A850000AD8B4BC
:10637000CEEF31F00101556B0001010155510001D3
:1063800067EC00F00009D8B4CEEF31F00101552BD5
:106390006E6F000173EC08F0BDEF31F04AEF39F099
:1063A000010120511408D8B403D00001F8EF31F0F6
:1063B0000001F0EC25F002C056F101C055F1120EBB
:1063C000A96E55C1A8FFA69CA69EA684F250006E99
:1063D000F29E0F01550EA76EAA0EA76EA6820001AF
:1063E000A6B2F0EF31F0A6940050F2124AEF39F065
:1063F000010120511508D8B403D00001DDEF32F0BF
:106400000001010E926E090EA96EA69CA69EA680A2
:10641000A850120F0101566F000156C157F1B4EC9C
:106420000DF001012C6B2B6B000102C02AF101C0A1
:1064300029F101011D6B000101011D510F08D8B0A8
:1064400003D000016AEF32F000012CC130F12BC102
:106450002FF12AC12EF129C12DF1350E01011D2583
:10646000E96E010EEA6ED8B0EA2A000130C15BF194
:106470002FC15AF12EC159F12DC158F101011D5101
:10648000576FD8A403D0000155EF32F00001D89027
:1064900001015B335A3359335833572F02D004D09C
:1064A0000001000147EF32F0000101015851010BDA
:1064B000006E5951000B016E5A51000B026E5B5178
:1064C000000B036E000100C0EFFF01011D2B000156
:1064D0001CEF32F0030E01011D6F000101011D517F
:1064E0000608D8B003D0000196EF32F00001350E57
:1064F00001011D25E96E010EEA6ED8B0EA2AEF52BD
:10650000D8A403D0000189EF32F00001310E8AEFE8
:1065100032F0300E0101556F000155C16EF173EC80
:1065200008F001011D2B00016EEF32F0000E81BA60
:10653000010E000AD8A4C8EF32F001011D6B000162
:1065400001011D510108D8B003D00001C8EF32F09D
:106550000001350E01011D25E96E010EEA6ED8B06D
:10656000EA2AEF52D8A403D00001BBEF32F00001B9
:10657000310EBCEF32F0300E0101556F000155C1F4
:106580006EF173EC08F001011D2B0001A0EF32F059
:1065900001013C53D8A403D00001D3EF32F0000135
:1065A000310ED4EF32F0300E0101556F000155C1AC
:1065B0006EF173EC08F04AEF39F001012051160832
:1065C000D8B403D0000111EF33F0000101011D6BBD
:1065D000000101011D510408D8B003D000010BEFE8
:1065E00033F00001320E01011D25E96EEA6AD8B0D0
:1065F000EA2A0001EFCF55F155C156F1C0EC26F063
:106600003A0E01016E6F000173EC08F001011D2BC1
:106610000001E9EF32F037C056F1C0EC26F04AEF46
:1066200039F0010120511B08D8B403D0000139EF23
:1066300033F00001F0EC25F002C026F101C025F195
:10664000F0EC25F002C028F101C027F1010E926E96
:1066500081EC03F028C155F10101566B000125C101
:106660005CF155C15DF127C15EF1D7EC03F04AEF53
:1066700039F0010120511C08D8B403D0000172EF99
:1066800033F000010101646B000124C063F150ECA0
:1066900012F02E0E01016E6F000173EC08F0010183
:1066A000646B000123C063F150EC12F02E0E010167
:1066B0006E6F000173EC08F00101646B000122C0F1
:1066C00063F150EC12F02E0E01016E6F000173ECBD
:1066D00008F00101646B000121C063F150EC12F07D
:1066E0004AEF39F0010120511D08D8B403D0000150
:1066F000ABEF33F000010101646B000128C063F1CE
:1067000050EC12F02E0E01016E6F000173EC08F0D8
:106710000101646B000127C063F150EC12F02E0EF2
:1067200001016E6F000173EC08F00101646B000160
:1067300026C063F150EC12F02E0E01016E6F0001C5
:1067400073EC08F00101646B000125C063F150ECAB
:1067500012F04AEF39F0010120511E08D8B403D0DD
:1067600000015DEF34F00001010E926E0101286B13
:10677000276B030E1D6F000101011D510608D8B0E3
:1067800003D00001E9EF33F00001F0EC25F002C086
:1067900026F101C025F126C103F001012551026E49
:1067A0001D51006ED8A403D00001DEEF33F00001CC
:1067B000D89002360336002ED8EF33F00250010194
:1067C000272703502823000101011D2B0001BCEFE6
:1067D00033F0000E81BA010E000AD8A420EF34F085
:1067E00001011D6B000101011D510108D8B003D04A
:1067F000000120EF34F00001F0EC25F002C026F19A
:1068000001C025F126C103F001012551026E1D5181
:10681000006ED8A403D0000115EF34F00001D89029
:1068200002360336002E0FEF34F002500101272705
:1068300003502823000101011D2B0001F3EF33F069
:10684000F0EC25F002C026F101C025F1010125354B
:10685000026E2635036E02360336023603360236E2
:106860000336023603360236033602360336800E0E
:1068700002160250272703502823040E2727FF0E55
:106880002823000181EC03F0090EA96EA69CA69EA8
:10689000A680A850120F0101566F000128C157F1C0
:1068A0000101586B000156C15CF157C15DF127C170
:1068B0005EF1D7EC03F04AEF39F0010120512008D6
:1068C000D8B403D000017CEF34F000010101556B16
:1068D0000001010155510001A8EC00F00009D8B4F5
:1068E0007AEF34F00101552B6E6F000173EC08F064
:1068F00069EF34F04AEF39F0010120512108D8B492
:1069000003D000019BEF34F000010101556B000141
:10691000010155510001BAEC00F00009D8B499EF1B
:1069200034F00101552B6E6F000173EC08F088EF15
:1069300034F04AEF39F0010120512208D8B403D0D5
:106940000001D7EF34F00001000E81BA010E000AF9
:10695000D8A4C1EF34F00101556B0001010155517C
:106960000001C7EC00F00009D8B4BFEF34F001011A
:10697000552B6E6F000173EC08F0AEEF34F0D5EFDD
:1069800034F00101556B0001010155510001D5ECB6
:1069900000F00009D8B4D5EF34F00101552B6E6F2B
:1069A000000173EC08F0C4EF34F04AEF39F0010154
:1069B00020512308D8B403D00001F6EF34F00001D1
:1069C0000101556B0001010155510001E3EC00F09C
:1069D0000009D8B4F4EF34F00101552B6E6F0001BB
:1069E00073EC08F0E3EF34F04AEF39F00101205185
:1069F0002A08D8B403D000010FEF35F00001020ED1
:106A0000A96EA69CA69EA680A8500101556F646B36
:106A1000000155C163F150EC12F04AEF39F0010169
:106A200020512B08D8B403D0000128EF35F0000125
:106A3000030EA96EA69CA69EA680A8500101556FC4
:106A4000646B000155C163F150EC12F04AEF39F06C
:106A5000010120512C08D8B403D0000141EF35F0DA
:106A60000001040EA96EA69CA69EA680A850010156
:106A7000556F646B000155C163F150EC12F04AEFA1
:106A800039F0010120512D08D8B403D000015AEF8C
:106A900035F00001050EA96EA69CA69EA680A85002
:106AA0000101556F646B000155C163F150EC12F0A8
:106AB0004AEF39F0010120512E08D8B403D000016B
:106AC00073EF35F00001130EA96EA69CA69EA6805A
:106AD000A8500101556F646B000155C163F150EC82
:106AE00012F04AEF39F0010120512F08D8B403D039
:106AF00000018CEF35F00001140EA96EA69CA69E35
:106B0000A680A8500101556F646B000155C163F167
:106B100050EC12F04AEF39F0010120513008D8B49E
:106B200003D00001A5EF35F00001150EA96EA69C5B
:106B3000A69EA680A8500101556F646B000155C147
:106B400063F150EC12F04AEF39F0010120513108A5
:106B5000D8B403D00001BEEF35F00001160EA96EC7
:106B6000A69CA69EA680A8500101556F646B0001EB
:106B700055C163F150EC12F04AEF39F00101205198
:106B80003208D8B403D00001D7EF35F00001170E5A
:106B9000A96EA69CA69EA680A8500101556F646BA5
:106BA000000155C163F150EC12F04AEF39F00101D8
:106BB00020513308D8B403D00001F0EF35F00001C4
:106BC000180EA96EA69CA69EA680A8500101556F1E
:106BD000646B000155C163F150EC12F04AEF39F0DB
:106BE000010120513408D8B403D0000109EF36F078
:106BF0000001190EA96EA69CA69EA680A8500101B0
:106C0000556F646B000155C163F150EC12F04AEF0F
:106C100039F0010120513508D8B403D0000122EF2A
:106C200036F000011A0EA96EA69CA69EA680A8505A
:106C30000101556F646B000155C163F150EC12F016
:106C40004AEF39F0010120513608D8B403D00001D1
:106C500036EF37F00001010E926E81EC03F0010176
:106C6000566B1B0E556F0001CFEC26F002C056F19B
:106C700001C055F155C157F1B4EC0DF001012C6B79
:106C80002B6B000102C02AF101C029F10A0E01019B
:106C90001D6F000101011D510D08D8B003D0000186
:106CA00098EF36F000012CC130F12BC12FF12AC131
:106CB0002EF129C12DF1350E01011D25E96E010EC0
:106CC000EA6ED8B0EA2A000130C15BF12FC15AF157
:106CD0002EC159F12DC158F101011D51576FD8A492
:106CE00003D0000183EF36F00001D89001015B333F
:106CF0005A3359335833572F02D004D000010001C2
:106D000075EF36F0000101015851010B006E595129
:106D1000000B016E5A51000B026E5B51000B036EAB
:106D2000000100C0EFFF01011D2B00014AEF36F00A
:106D30000101566B1B0E556F00013EEC27F002C09F
:106D400056F101C055F155C157F1B4EC0DF00101F8
:106D50002C6B2B6B000102C02AF101C029F11B0E24
:106D6000A96EA69CA69EA680A8500108D8B4D7EF0D
:106D700036F01B0EA96EA69CA69EA680A8500308FE
:106D8000D8B4D7EF36F01B0EA96EA69CA69EA6809F
:106D9000A8500608D8B4D7EF36F01B0EA96EA69CF3
:106DA000A69EA680A8500708D8A4E2EF36F02AC114
:106DB00029F12BC12AF12CC12BF101012C6B00010F
:106DC000EAEF36F0000E01012A17000E2B17000E15
:106DD0002C170001010129372A372B372C37293787
:106DE0002A372B372C3729372A372B372C37293797
:106DF0002A372B372C37F00E29174251080DF35044
:106E00002925556F000E2A21566F000E2B21576F32
:106E1000000E2C21586F4151040DF3505525596F28
:106E2000000E56215A6F000E57215B6F000E58213D
:106E30005C6FD8904035006E59255D6F000E5A2169
:106E40005E6F000E5B215F6F000E5C21606F3F5133
:106E50005D25616F000E5E21626F000162C164F109
:106E600061C163F150EC12F04AEF39F00101205199
:106E70003708D8B403D000014FEF37F000011B0EE4
:106E8000A96EA69CA69EA680A8500101556F646BB2
:106E9000000155C163F150EC12F04AEF39F00101E5
:106EA00020513808D8B403D0000177EF37F0000143
:106EB000F0EC25F002C056F101C055F11B0EA96E91
:106EC00055C1A8FFA69CA69EA684F250006EF29E15
:106ED0000F01550EA76EAA0EA76EA6820001A6B2DC
:106EE0006FEF37F0A6940050F2124AEF39F001012B
:106EF00020513908D8B403D00001BAEF38F00001AE
:106F0000010E926EF0EC25F001C041F11B0EA96E4E
:106F1000A69CA69EA680A8500808D8B49AEF37F081
:106F2000080EA96EA69CA69EA680A850000AD8A40A
:106F30009DEF37F00101416B0001F0EC25F002C03C
:106F400026F101C025F101012653D8B403D0000178
:106F5000B4EF37F00001010125510008D8A003D09B
:106F60000001B8EF38F00001010126510F08D8B038
:106F700003D00001B8EF38F0000126C128F125C187
:106F800027F1010127510F0B556F2851000B566F48
:106F9000276B5535286F2837FC0E2817566B1B0EAC
:106FA000556F0001CFEC26F002C056F101C055F13B
:106FB00055C157F1B4EC0DF001012C6B2B6B0001A6
:106FC00002C02AF101C029F101012999C30E2A1733
:106FD000000E2B17000E2C1727512925556F28510D
:106FE0002A21566F000E2B21576F000E2C21586F4F
:106FF0004139006EF00E001600505525296F000E25
:1070000056212A6F000E57212B6F000E58212C6F2E
:10701000000181EC03F00101566B1B0E556F00015E
:10702000CFEC26F002C056F101C055F12AC158F14B
:107030002BC159F12CC15AF101015B6B000155C103
:107040005CF158C15DF129C15EF1D7EC03F026C1B6
:1070500028F125C127F101012833273328332733AD
:1070600028332733283327330F0E28171B0EA96E1A
:10707000A69CA69EA680A8500108D8A403D0000113
:1070800061EF38F000011B0EA96EA69CA69EA6809B
:10709000A8500308D8B461EF38F01B0EA96EA69C67
:1070A000A69EA680A8500608D8B461EF38F01B0E43
:1070B000A96EA69CA69EA680A8500708D8A48BEF10
:1070C00038F00101566B1B0E556F00013EEC27F0A6
:1070D00002C056F101C055F155C157F1B4EC0DF0A5
:1070E00002C026F101C025F181EC03F00101566BCD
:1070F0001B0E556F00013EEC27F002C056F101C097
:1071000055F155C15CF127C15DF125C15EF1D7ECA8
:1071100003F0B8EF38F00101566B1B0E556F0001FC
:107120003EEC27F002C056F101C055F155C157F1B0
:10713000B4EC0DF002C026F101C025F181EC03F0A2
:107140000101566B1B0E556F00013EEC27F002C08B
:1071500056F101C055F126C157F10101586B0001EC
:1071600055C15CF157C15DF127C15EF1D7EC03F069
:107170004AEF39F0010120513A08D8B403D0000198
:1071800044EF39F00001010E926E81EC03F0010131
:10719000566B1B0E556F0001CFEC26F002C056F166
:1071A00001C055F155C157F1B4EC0DF001012C6B44
:1071B0002B6B000102C02AF101C029F101011D6BF6
:1071C000000101011D510F08D8B003D000012FEFBD
:1071D00039F000012CC130F12BC12FF12AC12EF161
:1071E00029C12DF1350E01011D25E96E010EEA6E52
:1071F000D8B0EA2A000130C15BF12FC15AF12EC18B
:1072000059F12DC158F101011D51576FD8A403D078
:1072100000011AEF39F00001D89001015B335A33B5
:1072200059335833572F02D004D0000100010CEF1E
:1072300039F0000101015851010B006E5951000B4A
:10724000016E5A51000B026E5B51000B036E000180
:1072500000C0EFFF01011D2B0001E1EF38F001013B
:107260003953D8A403D000013AEF39F00001310EB0
:107270003BEF39F0300E0101556F000155C16EF141
:1072800073EC08F04AEF39F03F0E01016E6F000118
:1072900073EC08F050EF39F01FC16EF173EC08F099
:1072A000B4EF28F0A7EF27F0010E016E5AEF39F086
:1072B000000E016E12EF3CF0080EAD6FAC6B299022
:1072C000C3C02AF0C4C02BF0B8C021F1B7C020F170
:1072D0001EEC15F0BAC021F1B9C020F11EEC15F07A
:1072E0000101216BCA0E206F0001B3EC14F0010103
:1072F000216BC60E206F0001B3EC14F001011E518A
:10730000020B000AD8A403D000018BEF39F0000172
:10731000600E8CEF39F0500E01011F6F00011FC18C
:107320006EF173EC08F01EC16EF173EC08F00B0EF9
:1073300001016E6F000173EC08F0B80E01016E6F71
:10734000000173EC08F001011E51020B000AD8A4E1
:1073500003D00001CFEF39F000010101216B280EAD
:10736000206F00018AEC14F0020E01016E6F000123
:1073700073EC08F0040E01016E6F000173EC08F06D
:10738000050E0101216FB40E206F00011EEC15F0F7
:107390000101216B240E206F00018AEC14F0010121
:1073A000216B190E206F000129EC15F00101216BF2
:1073B000B30E206F000129EC15F001016F6B000185
:1073C0004CEC08F0060E01016F6F00014CEC08F068
:1073D000140EC15D01011F6F000E0001C2590101B1
:1073E000206F000120C122F11FC121F1BEEC15F078
:1073F0002A5001011F6F1F1F00011FC16EF173ECA6
:1074000008F02B5001011F6F1F1F00011FC16EF1FB
:1074100073EC08F00101216B206B00011EEC15F0EC
:1074200001011E51020B000AD8A403D0000121EF74
:107430003AF000010101216B2C0E206F00018AEC53
:1074400014F055EF3AF021EC08F02AC0C3F02BC03D
:10745000C4F06E52D8A435EF3AF06D502708D8A08A
:1074600035EF3AF06E6A280E6D6E01011D51020B68
:10747000000AD8A403D0000143EF3AF00001040E43
:107480006D26000E6E226EC0C2F06DC0C1F001010B
:10749000216B206B00018AEC14F0060EAE6F60ECDD
:1074A00015F01DC11EF15CEF39F01DEC16F022EF56
:1074B0003CF0100E01011A6F29902B6A00012BC0BD
:1074C0002AF001011F6BB90E1E6F000107EC1BF0C3
:1074D0000152D8B426EF3CF001011F6BB70E1E6FAE
:1074E000000107EC1BF00152D8B426EF3CF001017B
:1074F0001E6BC60E1D6F000144EC1BF00152D8B488
:1075000026EF3CF001011E6BCA0E1D6F000144EC1A
:107510001BF00152D8B426EF3CF0010E0101686F58
:10752000180E676F000188EC0BF00152D8B426EFFB
:107530003CF0010E0101686F190E676F000188ECC5
:107540000BF00152D8B426EF3CF001011F6B060E80
:107550001E6F000193EC1BF00152D8B426EF3CF0F3
:10756000C253D8A4B9EF3AF0C1512708D8B026EFDA
:107570003CF01950AF5DD8A426EF3CF01A50B05D36
:10758000D8A426EF3CF01B50B15DD8A426EF3CF008
:107590001C50B25DD8A426EF3CF0140EC15D010171
:1075A0001D6F000E0001C25901011E6F00011EC1B6
:1075B00022F11DC121F1BEEC15F00101216B190E64
:1075C000206F000129EC15F00101216BB30E206F33
:1075D000000129EC15F001016F6B00014CEC08F083
:1075E000060E01016F6F00014CEC08F0010118510B
:1075F0005008D8A003D000011CEF3BF00001C1539C
:10760000D8A407EF3BF0C253D8B41CEF3BF0010104
:107610001F6B040E1E6F000193EC1BF00152D8B4D7
:107620001CEF3BF0040EC15F000EC25B100E0101A7
:10763000185F0001F6EF3AF0280EC15DD06F000E22
:10764000C259D16F3FC01CF13EC01BF1D1C01FF128
:10765000D0C01EF193EC1BF01CC11FF11BC11EF129
:1076600041EC1EF02A3C26EF3CF02B3C26EF3CF090
:1076700001011D6B0001D1EC1AF00101216B280EF4
:10768000206F00018AEC14F0C46BC4C0C3F02996CB
:107690002994298801011951040B000AD8A403D0A8
:1076A000000159EF3BF0000101011A6B000116EFD8
:1076B0003CF001011951020B000AD8A403D00001CB
:1076C00098EF3BF000010101206BC60E1F6F226B8B
:1076D000010E216F000198EC22F0B7510D08D8A4DB
:1076E00076EF3BF0B853D8B47FEF3BF0B75150087A
:1076F000D8A492EF3BF0B853D8A492EF3BF0FF0E22
:10770000CB6FFF0ECA6FCF51036ECE51CE2BD8B4C4
:10771000CF2BCC6F03C0CDF0120E01011A6F000108
:1077200096EF3BF0140E01011A6F000116EF3CF0CA
:1077300001011951010B000AD8A403D00001B7EFD1
:107740003BF00001010ED02501011D6F000E00016C
:10775000D12101011E6F206BC60E1F6F00011EC1DB
:1077600022F11DC121F198EC22F016EF3CF001014D
:107770001951100B000AD8A403D0000116EF3CF0F9
:107780000001D051D111D8B4D3EF3BF00101206BEF
:10779000C60E1F6F0001D1C022F1D0C021F198ECBC
:1077A00022F0D6EF3BF001011A6B0001B7510D0832
:1077B000D8A402EF3CF0B853D8A402EF3CF0CA536F
:1077C000D8A402EF3CF0CB53D8A402EF3CF0010167
:1077D0001D6B000101011D51000130EC00F00101A1
:1077E0001D2B6D6F00019FEC08F00C0E01011D5D5B
:1077F000D8B403D00001EAEF3BF0110E1A6F00017C
:1078000016EF3CF0B7515008D8A416EF3CF0B8532F
:10781000D8A416EF3CF0D051D111D8B416EF3CF0FB
:10782000B8EF27F0110E01011A6F000101011A5380
:10783000D8A403D0000122EF3CF000011AC11DF1D1
:1078400023EF3AF0010E016E28EF3CF0000E016EBE
:107850002DEF3FF0F86AD08EFE0E006E050E016E21
:10786000EA6A020EE96EEF6AE92AD8B4EA2A002E23
:1078700033EF3CF0012E33EF3CF0EA6AE96A070E81
:10788000C16E056A066A010E076E086A096A0A6A0D
:107890000B6A810EAF6E260EAC6E900EAB6E156A43
:1078A000166A060E186E326A400E336EF60E346E8D
:1078B000FD0E356E366A376AC56BEC6B0101156BD0
:1078C000166B0001F29CF29EF2BE63EF3CF0130EC9
:1078D000926E826AFF0E946EFF0E956E8480848293
:1078E0008484969096929694000E80B8010E000AB9
:1078F000D8A4E8EF3CF0140E0101186F0001FA0E55
:107900000101646F0001C6EC01F00101182F02D0E3
:1079100003D000010001F3D7000E80B8010E000A69
:10792000D8B403D00001E8EF3CF00001A96AA69C9E
:10793000A69EA680A850366E010EA96EA69CA69E95
:10794000A680A850376E01011B6B190E1A6FC00E6E
:107950001C6FA80E1D6F1E6B020E1F6F0001DCEC6A
:1079600001F001011B6B210E1A6FFF0E1C6FFF0E41
:107970001D6FFF0E1E6F1F6B0001DCEC01F001019B
:107980001B6B250E1A6FC00E1C6FA80E1D6F1E6B91
:10799000010E1F6F0001DCEC01F024EC02F0120E6E
:1079A000A96E010EA86EA69CA69EA684F250006E3B
:1079B000F29E0F01550EA76EAA0EA76EA6820001B9
:1079C000A6B2E0EF3CF0A6940050F2129AEC05F05B
:1079D000F19ECF6AB50ECD6ECD9E0101216B120EC8
:1079E000206F236B226B000136EC07F01486149A8B
:1079F000149880848086298629842998FE0E946EA6
:107A00008B808B901E0E0101646F0001C6EC01F0AB
:107A1000640E0101646F0001C6EC01F08B801E0E44
:107A20000101646F0001C6EC01F0FF0E946E0101CC
:107A3000186B00010101185100011CEC01F001015B
:107A4000182B00019EA822EF3DF0AD6E040E01013F
:107A5000185DD8B403D000011AEF3DF0000E81BAD2
:107A6000010E000AD8B403D0000152EF3DF000012E
:107A70000101186B0001010118510001C7EC00F071
:107A80000101182B00019EA843EF3DF0AD6E0A0ED8
:107A90000101185DD8B403D000013BEF3DF00001B7
:107AA0006AEF3DF00101186B00010101185100015E
:107AB000D5EC00F00101182B00019EA85DEF3DF010
:107AC000AD6E0A0E0101185DD8B403D0000155EF68
:107AD0003DF00001200E01016D6F00019FEC08F0E8
:107AE0000101186B000101011851000127EC01F0A0
:107AF0000101182B6D6F00019FEC08F00F0E0101C2
:107B0000185DD8B403D0000173EF3DF0030E196F78
:107B10000001390E01016D6F00019FEC08F00101B9
:107B2000192F02D004D00001000189EF3DF0200E92
:107B30006D6F00019FEC08F00101186B000101015D
:107B400018510001BAEC00F00101182B6D6F000113
:107B50009FEC08F0080E0101185DD8B403D00001B5
:107B60009FEF3DF00A0E6D6F00019FEC08F0BFEC37
:107B700008F00152D8A435EF3EF00101186B000166
:107B800001011851000137EC01F00101182B6D6F54
:107B900000019FEC08F0070E0101185DD8B403D076
:107BA0000001C0EF3DF0000196EF0CF00A0EA96E47
:107BB000310EA86EA69CA69EA684F250006EF29E80
:107BC0000F01550EA76EAA0EA76EA6820001A6B2DF
:107BD000E7EF3DF0A6940050F2120B0EA96E320EA4
:107BE000A86EA69CA69EA684F250006EF29E0F017F
:107BF000550EA76EAA0EA76EA6820001A6B2FEEFD2
:107C00003DF0A6940050F2120C0EA96E330EA86E31
:107C1000A69CA69EA684F250006EF29E0F01550E01
:107C2000A76EAA0EA76EA6820001A6B215EF3EF0BF
:107C3000A6940050F212120EA96EA86AA69CA69EE7
:107C4000A684F250006EF29E0F01550EA76EAA0E8A
:107C5000A76EA6820001A6B22BEF3EF0A6940050BC
:107C6000F2129AEC05F0B7EF3DF058EF0FF0E1ECAF
:107C700010F0120EA96EA69CA69EA680A850176EA4
:107C80001752D8A44AEF3EF01C6A1B6A1A6A196A96
:107C900055EF3EF0148EBFEC08F0A4EC12F0ECECC3
:107CA00012F034EC13F07CEC13F00D0E9EA856EF9E
:107CB0003EF0AD6E0A0E9EA85BEF3EF0AD6E090E73
:107CC000A96E020EA86EA69CA69EA684F250006E17
:107CD000F29E0F01550EA76EAA0EA76EA682000196
:107CE000A6B270EF3EF0A6940050F2121B0EA96EE1
:107CF000010EA86EA69CA69EA684F250006EF29E6F
:107D00000F01550EA76EAA0EA76EA6820001A6B29D
:107D100087EF3EF0A6940050F212000E80B8010EDC
:107D2000000AD8A4CDEF3EF00D0E9EA895EF3EF0D0
:107D3000AD6E0A0E9EA89AEF3EF0AD6E0101176B74
:107D40000001010117513F08D8B003D00001CCEF6A
:107D50003EF0000117C157F1B4EC0DF002C019F16B
:107D600001C018F119C11FF1370E0101206F000188
:107D70007AEC0DF018C11FF1370E0101206F0001E0
:107D80007AEC0DF0200E9EA8C3EF3EF0AD6E01011F
:107D9000172B0001A1EF3EF08088ADEC09F01752DF
:107DA000D8A4DAEF3EF01850165CD8B0DAEF3EF007
:107DB00065EF18F01752D8A4F0EF3EF01850165C9B
:107DC000D8A0F0EF3EF0148EBFEC08F0A4EC12F057
:107DD000ECEC12F034EC13F07CEC13F0010E176EA7
:107DE000D3EF19F00152D8B42FEF3FF001011D6B12
:107DF0000001D1EC1AF0AC510608D8A407EF3FF00F
:107E0000AD510808D8A407EF3FF07CEF1CF0AC534D
:107E1000D8A42DEF3FF0AD510808D8A42DEF3FF0C6
:107E200092EF1DF00152D8B42DEF3FF0AE2D1DEFB3
:107E30003FF0F5EF1EF02DEF3FF0AE511108D8A442
:107E400026EF3FF09BEF21F02DEF3FF0AE510608FB
:107E5000D8A42DEF3FF059EF3AF03D6A3C6A152C5B
:0C7E600033EF3FF0FF008DEF3EF0030019
:020000040030CA
:0C000000FFFAFCFEFFFFFBFFFFFFFFFF0D
:00000001FF
